:100000000C94FC000C9424010C9424010C94240105
:100010000C9424010C9424010C9424010C942401CC
:100020000C9424010C9424010C9419160C94921530
:100030000C94C8160C9424010C9424010C942401F3
:100040000C94AC2A0C9424010C94952C0C941F2D28
:100050000C9424010C9424010C9424010C9424018C
:100060000C94CF100C942401253032643A253032A0
:10007000643A253032642E253033753B00504F539F
:100080004D534B2C00504F534D534F2C53746F70A6
:10009000204E4D4541204C6F6767657200504F53AD
:1000A0004D53542C5374617274204E4D4541204C75
:1000B0006F676765722C5620302E312E3135006403
:1000C000617461303030302E64617400504F534D94
:1000D0004346472C25752C25752C25752C25752C0C
:1000E00025782C257500504F534D534F2C52656188
:1000F000736F6E3A2074696D657320757000504F90
:10010000534D534F2C526561736F6E3A2073746F69
:10011000702073776974636800504F534D534F2CB0
:10012000526561736F6E3A20737570706C79206CD4
:100130006F7700504F534D4143432C25692C25695F
:100140002C256900504F534D4759522C25692C25B9
:10015000692C256900504F534D5643432C25692C7B
:10016000256900636F6E6669672E646174005620AE
:10017000302E312E3135006F7365616D6C6F672ED7
:10018000636E66007C3C3E5E2B3D3F2F5B5D3B2CEF
:100190002A225C0000000000240027002A00000042
:1001A0000000250028002B0000000000230026008E
:1001B00029000404040404040404020202020202EA
:1001C000030303030303010204081020408001021B
:1001D000040810200102040810200000000700029B
:1001E00001000003040600000000000000004505B7
:1001F0006B0FB0174D303E0511241FBECFEFD8E076
:10020000DEBFCDBF11E0A0E0B1E0E0E4F7E602C060
:1002100005900D92A236B107D9F717E0A2E6B1E03A
:1002200001C01D92A332B107E1F711E0C6EFD1E0A2
:1002300004C02297FE010E944D33CE3ED107C9F77C
:100240000E948B300C9493330C940000A0E0B0E03B
:10025000ECE2F1E00C945D33EC012B016A016115D5
:10026000710519F0FB0191838083C114D10449F019
:10027000C6010297839728F020E030E040E050E08C
:10028000DCC0A9908A2D90E00E945133892BC9F7D8
:10029000FDE2AF1621F4A9903324339405C08BE21C
:1002A000A81609F4A9903324C114D10421F0E0E187
:1002B000CE16D10411F5F0E3AF1669F488818837C2
:1002C00011F0883541F4A980229682E0382A20E195
:1002D000C22ED12C12C0C114D10479F4E0E3AE16C1
:1002E00059F199E9E92E99E9F92E99E9092F99E14E
:1002F000192F8AE0C82ED12C3AC0FAE0CF16D104CB
:1003000091F080E1C816D10429F0E8E0CE16D104BE
:10031000F9F415C0BFEFEB2EBFEFFB2EBFEF0B2F95
:10032000BFE01B2F24C0A9E9EA2EA9E9FA2EA9E90A
:100330000A2FA9E11A2F1BC0F8E0CF2ED12CEFEF26
:10034000EE2EEFEFFE2EEFEF0E2FEFE11E2F0FC080
:100350009601442737FD4095542F6FEF7FEF8FEFC5
:100360009FEF0E940E33C901DA017C018D0120E06C
:1003700030E040E050E060E03601882477FC809473
:10038000982C70EDB72EBA0CF9E0FB1570F48A2D9D
:1003900081548A3118F499ECB92E06C08A2D815601
:1003A0008A3148F589EAB82EBA0C8B2D90E08C156D
:1003B0009D050CF56F3FE9F0E216F30604071507FB
:1003C000B8F0CA01B901A40193010E94C8329B018F
:1003D000AC018B2D90E0A0E0B0E0280F391F4A1F40
:1003E0005B1F281739074A075B0710F061E001C05F
:1003F0006FEFA990C6CF4114510451F0662311F05C
:10040000219703C031FE04C02297F201D183C0833B
:1004100030FE07C050954095309521953F4F4F4F86
:100420005F4F67FF0AC082E290E0909322078093BB
:1004300021072FEF3FEF4FEF5FEFB901CA01CDB7B3
:10044000DEB7E1E10C947933FB01DC0105900D92FC
:100450000020E1F70895FB01DC0104C08D910190BB
:10046000801921F441505040C8F7881B990B08951A
:10047000FB01DC0102C001900D9241505040D8F7C1
:100480000895FB01DC0101900D920020E1F7089531
:10049000AEE0B0E0EEE4F2E00C946A330D891E8920
:1004A0008EE08C831A8309838FEF9FE79E838D8371
:1004B0009E01275E3F4FCE0101966F89788DA9017D
:1004C0000E946C022F813885020F131FF8011082E1
:1004D0002E96E4E00C948633ABE0B0E0E2E7F2E085
:1004E0000C945C333C012B015A01FC0117821682EB
:1004F000838181FD03C06FEF7FEFC6C19AE0892E33
:100500001E010894211C311CF3012381F20123FDFB
:10051000859123FF81912F01882309F4B2C185328F
:1005200039F423FD859123FF81912F01853229F430
:1005300090E0B3010E945F04E7CF982FFF24EE24E0
:100540009924FFE1FF15D0F09B3269F09C3228F42A
:10055000903259F0933291F40EC09D3249F09033AD
:1005600069F441E024C052E0F52A84E0F82A28C06A
:1005700098E0F92A25C0E0E1FE2A22C0F7FC29C054
:10058000892F80538A3070F4F6FE05C0989C902C19
:100590001124980E15C0E89CE02C1124E80EF0E21E
:1005A000FF2A0EC09E3229F4F6FC6BC140E4F42A07
:1005B00007C09C3619F450E8F52A02C0983649F471
:1005C000F20123FD959123FF91912F01992309F0C9
:1005D000B8CF892F8554833018F08052833038F497
:1005E00044E050E0A40EB51E5FE359830FC093367C
:1005F00031F0933779F0933509F056C020C0F501FA
:100600008081898342E050E0A40EB51E610101E0C3
:1006100010E012C0F501C080D180F6FC03C06FEF7E
:100620007FEF02C0692D70E042E050E0A40EB51EDD
:10063000C6010E9454048C015FE7F52214C0F50145
:10064000C080D180F6FC03C06FEF7FEF02C0692D40
:1006500070E042E050E0A40EB51EC6010E944904BD
:100660008C0150E8F52AF3FE07C01AC080E290E042
:10067000B3010E945F04EA948E2D90E008171907D9
:10068000A8F30EC0F601F7FC8591F7FE81916F018A
:1006900090E0B3010E945F04E110EA940150104021
:1006A0000115110579F7EAC0943611F0993669F50C
:1006B000F7FE08C0F501208131814281538184E039
:1006C00090E00AC0F501808191819C01442737FDAB
:1006D0004095542F82E090E0A80EB91E9FE6F922C3
:1006E00057FF09C050954095309521953F4F4F4F8A
:1006F0005F4FE0E8FE2ACA01B901A1012AE030E01B
:100700000E948B04D82ED21840C0953729F41F2D93
:100710001F7E2AE030E01DC01F2D197F9F3661F03B
:10072000903720F4983509F0ACC00FC0903739F0FD
:10073000983709F0A6C004C028E030E00AC0106174
:1007400014FD146020E130E004C014FD166020E1C7
:1007500032E017FF08C0F5016081718182819381C9
:1007600044E050E008C0F50180819181BC0180E047
:1007700090E042E050E0A40EB51EA1010E948B045F
:10078000D82ED2188FE7F82EF122F6FE0BC05EEFBE
:10079000F522D91438F4F4FE07C0F2FC05C08FEE40
:1007A000F82202C01D2D01C0192DF4FE0DC0FE015E
:1007B000ED0DF11D8081803319F499EEF92208C006
:1007C0001F5FF2FE05C003C08F2D867809F01F5F02
:1007D0000F2DF3FC14C0F0FE0FC01E1510F09D2C61
:1007E0000BC09D2C9E0C911A1E2D06C080E290E03D
:1007F000B3010E945F041F5F1E15C0F304C01E15E5
:1008000010F4E11A01C0EE2404FF0FC080E390E071
:10081000B3010E945F0402FF1DC001FD03C088E711
:1008200090E00EC088E590E00BC0802F867891F0B4
:1008300001FF02C08BE201C080E2F7FC8DE290E094
:10084000B3010E945F0406C080E390E0B3010E9400
:100850005F049A94D914C0F3DA94F101ED0DF11DFF
:10086000808190E0B3010E945F04DD20A9F706C0FB
:1008700080E290E0B3010E945F04EA94EE20C1F7A9
:1008800043CEF30166817781CB012B96E2E10C9494
:100890007833FC010590615070400110D8F78095C5
:1008A00090958E0F9F1F0895FC016150704001903C
:1008B0000110D8F7809590958E0F9F1F08950F9384
:1008C0001F93CF93DF938C01EB018B8181FF1BC0C2
:1008D00082FF0DC02E813F818C819D8128173907B1
:1008E00064F4E881F9810193F983E88306C0E8851F
:1008F000F985802F0995892B31F48E819F8101968E
:100900009F838E8302C00FEF1FEFC801DF91CF914D
:100910001F910F910895FA01AA27283051F1203133
:1009200081F1E8946F936E7F6E5F7F4F8F4F9F4F83
:10093000AF4FB1E03ED0B4E03CD0670F781F891FC5
:100940009A1FA11D680F791F8A1F911DA11D6A0F93
:10095000711D811D911DA11D20D009F468943F9146
:100960002AE0269F11243019305D3193DEF6CF0145
:100970000895462F4770405D4193B3E00FD0C9F70B
:10098000F6CF462F4F70405D4A3318F0495D31FD78
:100990004052419302D0A9F7EACFB4E0A6959795CB
:1009A000879577956795BA95C9F7009761057105A1
:1009B00008959B01AC010A2E0694579547953795EB
:1009C0002795BA95C9F7620F731F841F951FA01D45
:1009D00008958130910509F03FC06F5F7F4F09F0A6
:1009E0004CC089E093E060E071E00E94A83289E1A8
:1009F0008093630110926601109279011092800138
:100A00001092820110929E011092A00110929D01FD
:100A100010929C018AE491E090939B0180939A014B
:100A20001092BD011092BC0188EE93E0A0E0B0E00E
:100A30008093BE019093BF01A093C001B093C10108
:100A400082E391E09093BB018093BA0187EC91E03F
:100A500068E60E9448140895892B79F46F5F7F4FF0
:100A600061F482E391E09093BB018093BA010E940C
:100A70003C1589E093E00E94C132089580E090E047
:100A80006FEF7FEF0E94E904089581E090E06FEF3F
:100A90007FEF0E94E90408951F93CF93DF93EC0149
:100AA0000E94F42A6093F4017093F5018093F6019B
:100AB0009093F7015E9ADE010D900020E9F71197FF
:100AC000AC1BBD0B10E090E005C0EC0FFD1F80815A
:100AD00018279F5FE92FF0E0EA17FB07B0F38AE9D8
:100AE00091E064E20E9455238AE991E0BE010E94F0
:100AF00029328AE991E06AE20E945523103128F4F4
:100B00008AE991E060E30E9455238AE991E0612F30
:100B100040E150E00E94AC31DF91CF911F910895E8
:100B20000F931F93682F0AE911E0C8010E94C43097
:100B3000C8016BE30E94C4301F910F9108956F921A
:100B40007F928F929F92AF92BF92CF92DF92EF925D
:100B5000FF920F931F936B017C0128EE33E040E07E
:100B600050E00E940E33B22EA32E942E852E8DB708
:100B70009EB70C970FB6F8949EBF0FBE8DBF0DB7F2
:100B80001EB70F5F1F4F84EF682E82E0782EEDB7FF
:100B9000FEB77282618288E690E0F80193838283D7
:100BA000622F732F842F952F20E13EE040E050E02C
:100BB0000E943033CA01B90128E130E040E050E042
:100BC0000E943033F801648315826B2D7A2D892DB4
:100BD000982D2CE330E040E050E00E943033CA0111
:100BE000B9012CE330E040E050E00E943033F801DE
:100BF000668317826B2D7A2D892D982D2CE330E09A
:100C000040E050E00E943033F80160871186C70150
:100C1000B60128EE33E040E050E00E940E33F801C8
:100C2000738762870E9448028DB79EB70C960FB6F5
:100C3000F8949EBF0FBE8DBF8AE991E0B3010E9478
:100C400029321F910F91FF90EF90DF90CF90BF90CE
:100C5000AF909F908F907F906F900895DF92EF926A
:100C6000FF920F931F93CF93DF937B018C01D42EC0
:100C7000E9018091A001882351F0C801B7010E94C9
:100C80009F058D2D0E949005CE010E944C05DF919D
:100C9000CF911F910F91FF90EF90DF9008950F93E8
:100CA0001F938091B9018823C9F18DB79EB708972A
:100CB0000FB6F8949EBF0FBE8DBFEDB7FEB731964D
:100CC00004EA12E0ADB7BEB712961C930E931197CB
:100CD00085E591E0938382838091F2019091F30105
:100CE000958384838091E9019091EA0197838683BB
:100CF0000E9448028DB79EB708960FB6F8949EBF23
:100D00000FBE8DBF6091F8017091F9018091FA01D9
:100D10009091FB0149E498010E942E061F910F91CA
:100D200008951F93CF93DF9380910601882309F4E0
:100D30006EC01092070311E057C08091D70188233D
:100D400051F40E94F42A6093000270930102809390
:100D50000202909303025D9ACA3019F410930703BC
:100D60000CC0CD3051F08091D701E82FF0E0EC5A63
:100D7000FD4FC0838F5F8093D70180910703882345
:100D800021F48091D701803578F18091D7018823B3
:100D900059F18091A001882329F10E94F42A6093DF
:100DA000F4017093F5018093F6019093F7015E9A38
:100DB0006091000270910102809102029091030201
:100DC0000E949F0582E40E9490054091D7018AE924
:100DD00091E064E572E050E00E946E238AE991E0C0
:100DE0000E94CC301092D7018AEB91E00E94391713
:100DF0001816190664F480910703882341F48AEBDE
:100E000091E00E940F17EC01992374F396CFDF91C4
:100E1000CF911F9108959091D60180910803981762
:100E200009F04AC084EA92E06DE770E00E94240273
:100E300020E02FC0E22FF0E0EC5FFD4F3081832FE8
:100E400082958F708A3018F4982F905D02C0982F89
:100E5000995CA4EAB2E0FD0131968C91882311F0EF
:100E6000DF01F9CF9C931082E32FEF70EA3018F482
:100E70009E2F905D02C09E2F995CA4EAB2E0FD0116
:100E800031968C91882311F0DF01F9CF9C93108269
:100E90002F5F8091D601281768F26091FC01709154
:100EA000FD018091FE019091FF0141E424EA32E0CE
:100EB0000E942E061092D60108951F93CF93DF93C0
:100EC00080910501882309F49BC01092060311E06C
:100ED00084C08091D601882351F40E94F42A609343
:100EE000FC017093FD018093FE019093FF015C9AD9
:100EF0008091B801882349F1D0FF10C00E940B07F0
:100F0000109306031092D6010E94F42A6093FC010C
:100F10007093FD018093FE019093FF019091D601A3
:100F2000913039F49E012F70822F8D5F80930803DA
:100F300003C0903508F051C0E92FF0E0EC5FFD4FA1
:100F4000C0839F5F9093D60148C0CA3019F41093B4
:100F500006030CC0CD3051F08091D601E82FF0E0AF
:100F6000EC5FFD4FC0838F5F8093D60180910603B5
:100F7000882321F48091D601803578F18091D601C3
:100F8000882359F18091A001882329F10E94F42A35
:100F90006093F4017093F5018093F6019093F7014B
:100FA0005E9A6091FC017091FD018091FE0190912B
:100FB000FF010E949F0581E40E9490054091D601A7
:100FC0008AE991E064E072E050E00E946E238AE9D1
:100FD00091E00E94CC301092D60188EF96E00E94FA
:100FE000152F1816190664F480910603882341F41E
:100FF00088EF96E00E946F2FEC01992374F369CF7C
:10100000DF91CF911F91089584EA92E065E870E046
:101010000E9424020E94F42A49E424EA32E00E9459
:101020002E068091A001882321F08EE991E00E9494
:10103000891D0895EF92FF920F931F938EE4809382
:101040007C0062E070E080E090E00E943D2B8091A7
:101050007A00806480937A0080917A0086FDFCCFCC
:101060008091780090E0A0E0B0E020917900F22E2D
:10107000EE240027F7FC0095102FE82AF92A0A2B06
:101080001B2B0E94F42A6093F8017093F90180935E
:10109000FA019093FB0160E070E381E190E0A80128
:1010A00097010E943033C9011F910F91FF90EF907B
:1010B00008950F931F930EE911E0C8010E94891D46
:1010C000C80168ED71E047E20E94E3221F910F9191
:1010D00008958F929F92AF92BF92CF92DF92EF923C
:1010E000FF920F931F93DF93CF9300D000D0CDB723
:1010F000DEB70E94F42A6B017C018CE496E060E18B
:1011000070E00E948328882E8CE496E061E170E014
:101110000E948328982E8CE496E062E170E00E94A1
:101120008328A82E8CE496E063E170E00E94832877
:10113000B82E19821A821B821C82FE01319624E18C
:1011400030E0AE014C5F5F4FF999FECF32BD21BD5B
:10115000F89A80B580832F5F3F4FE417F50711F0B1
:101160003196F2CF8CE496E069E170E00E9483282A
:101170002DB73EB7225130400FB6F8943EBF0FBE98
:101180002DBFEDB7FEB7319604EA12E0ADB7BEB79A
:1011900012961C930E9311972CEC30E0338322832C
:1011A0008482158296821782A0861186B286138663
:1011B00029813A814B815C8124873587468757870F
:1011C000808B118A0E9448022DB73EB72E5E3F4F9A
:1011D0000FB6F8943EBF0FBE2DBFC701B60149E45C
:1011E00098010E942E060F900F900F900F90CF91B4
:1011F000DF911F910F91FF90EF90DF90CF90BF9004
:10120000AF909F908F900895AF92BF92CF92DF9250
:10121000EF92FF920F931F93CF93DF930E940408E6
:101220008BB18F708BB900EF12C08BB180278BB957
:1012300064EF71E080E090E00E943D2B8BB180274D
:101240008BB964EF71E080E090E00E943D2B82E674
:1012500091E06AE044E00E942D23882331F388ED79
:1012600091E06FEB70E00E9424028BB18F708BB91C
:10127000C0910403D0910503219638E1A32E3CEFE1
:10128000B32E2CE9C22E2FEFD22E96EFE92E9FEF30
:10129000F92E6BC08BB180588BB9CE0168EE73E02C
:1012A0000E94E732262F205D2093DC016A9DF00129
:1012B0006B9DF00D7A9DF00D1124EC0FFD1FCF01F9
:1012C00064E670E00E94E732262F205D2093DD0166
:1012D0006C9D80016D9D100D7C9D100D11240E0FD5
:1012E0001F1FC8016AE070E00E94E732262F205DD0
:1012F0002093DE016E9DC0016F9D900D7E9D900D2F
:101300001124800F911F805D8093DF0182E691E0C0
:1013100068ED71E00E940E23882331F587E691E0A5
:101320000E9493258B019C0160916B0180E090E20B
:1013300070E00E94FB32882777FD8095982F061772
:1013400017072807390760F08EE991E068ED71E032
:1013500043E60E94E322D0930503C09304030AC02E
:1013600081E08093C60106C0219637E2C031D307E1
:1013700008F490CF84EA92E06DE970E00E942402C4
:101380000E94F42A49E424EA32E00E942E060E94D8
:101390006908DF91CF911F910F91FF90EF90DF903F
:1013A000CF90BF90AF900895CF92DF92EF92FF92CF
:1013B0000F931F9380910701882309F486C00E9430
:1013C000F42A6B017C0187EC91E06CEE71E04EEE4B
:1013D00051E020EF31E00E944B148DB79EB70A9781
:1013E0000FB6F8949EBF0FBE8DBFEDB7FEB7319616
:1013F00004EA12E0ADB7BEB712961C930E93119794
:1014000084E491E0938382838091EC019091ED01DB
:10141000958384838091EE019091EF019783868379
:101420008091F0019091F101918780870E9448029C
:101430008DB79EB70A960FB6F8949EBF0FBE8DBFAC
:10144000C701B60149E498010E942E0687EC91E09D
:101450006CEE71E04EEE51E020EF31E00E948F140F
:10146000ADB7BEB71A970FB6F894BEBF0FBEADBFEB
:10147000EDB7FEB7319612961C930E93119783E346
:1014800091E0938382838091EC019091ED019583AB
:1014900084838091EE019091EF0197838683809100
:1014A000F0019091F101918780870E9448028DB7E9
:1014B0009EB70A960FB6F8949EBF0FBE8DBFC701A8
:1014C000B60149E498010E942E061F910F91FF90EA
:1014D000EF90DF90CF900895EF92FF920F931F93BC
:1014E0000E94F42A7B018C018091C601882379F047
:1014F000C801B70124EF31E040E050E00E943033F2
:101500006B3F71058105910514F05F9801C05F9AEA
:101510008091F4019091F501A091F601B091F7014D
:101520008C599F4FAF4FBF4F8E159F05A007B10736
:1015300008F45E988091FC019091FD01A091FE015C
:10154000B091FF018C509E4FAF4FBF4F8E159F053E
:10155000A007B10708F45C98809100029091010205
:10156000A0910202B09103028C509E4FAF4FBF4F2B
:101570008E159F05A007B10708F45D980E941A0810
:101580009093F3018093F2012091E9013091EA01F7
:101590008217930730F083E00E94382C892B09F0E2
:1015A00095C08BB18F708BB98091A001882309F110
:1015B0000E944F062091F2013091F3018091E901E0
:1015C0009091EA012817390728F484EA92E069E14A
:1015D00071E004C084EA92E06EEF70E00E942402A1
:1015E0000E94F42A49E424EA32E00E942E060E9476
:1015F00004088BB1806F8BB960E177E280E090E006
:101600000E943D2B69C00E9404090E945D070E9450
:101610009106A8019701285E3340404050408091D8
:10162000E5019091E601A091E701B091E8018217F0
:101630009307A407B50708F04FC0E092E501F092C8
:10164000E6010093E7011093E8010E94D4090E948B
:101650004F06C801B70120E83EEE46E350E00E9485
:1016600030338091EB0190E082179307A8F484EA6D
:1016700092E066EE70E00E9424020E94F42A49E49F
:1016800024EA32E00E942E060E9404098091EB01B8
:101690008F5F8093EB0120C0C801B70120E63AEECE
:1016A00040E050E00E943033CA01B90120E031E04F
:1016B00040E050E00E943033162F8091030318174A
:1016C00059F00E9459081093030306C08091A001AD
:1016D000882309F09ACF97CF1F910F91FF90EF9039
:1016E00008956F927F928F929F92AF92BF92CF9206
:1016F000DF92EF92FF920F931F93F82E762E642EB7
:101700004801590188ED91E067E771E00E942402E9
:1017100082E691E068ED71E00E940E23882331F0AB
:1017200082E691E068ED71E00E940A238EE991E083
:1017300068ED71E043E60E94E3228091B8018823BE
:1017400029F08AE991E063E70E94C4308AE991E0D8
:101750006F2D4AE050E00E94AC318AE991E0672D9C
:101760004AE050E00E94AC318AE991E0662D4AE0FF
:1017700050E00E94AC3188ED91E06EE671E00E948D
:1017800024028AE991E068ED71E00E942C328AE936
:1017900091E0B501A40120E130E00E947B3160912D
:1017A000E9017091EA018AE991E04AE050E00E9483
:1017B0000A328AE991E06E2D4AE050E00E94AC3195
:1017C0008AE991E0B60140E150E00E948F318EE954
:1017D00091E00E94891D1F910F91FF90EF90DF9083
:1017E000CF90BF90AF909F908F907F906F90089513
:1017F0006F927F929F92AF92BF92CF92DF92EF92C1
:10180000FF920F931F93DF93CF9300D000D0CDB7FB
:10181000DEB788ED91E063E671E00E9424028CE47B
:1018200096E060E170E00E948328F82E8CE496E058
:1018300061E170E00E948328B82E8CE496E062E1BA
:1018400070E00E948328982E8CE496E063E170E0BB
:101850000E948328A82E19821A821B821C82FE01F4
:10186000319624E130E0AE014C5F5F4FF999FECF35
:1018700032BD21BDF89A80B580832F5F3F4FE417BA
:10188000F50711F03196F2CF8CE496E069E170E053
:101890000E948328E82E8AE08E1548F48CE496E0B6
:1018A00069E170E041E00E948A28EE24E394E0E0E0
:1018B000FEE7CC24CA94DC2C8491C8268C2D82951A
:1018C0008C25082E869586958025082E8695802560
:1018D00087700C2CCD2C869507948795D02CC82624
:1018E00006948795D024C826319680E8E030F80722
:1018F00019F78DEFC81687EBD80661F482E0E81679
:1019000049F08CE496E069E170E042E00E948A28A8
:1019100082E0E82E1092B80186E08F1510F403E003
:10192000F02E84E08B1510F413E0B12E85E08915BC
:1019300038F01092B801992019F081E08093B80135
:1019400082E691E068ED71E00E940E23882309F49D
:10195000EAC08EE991E068ED71E041E00E94E32287
:10196000882309F4E0C0109205011092060101E0FD
:1019700010E03E010894611C711CBBC08EE991E02F
:101980000E94C21E8D3011F08A3029F4112309F40F
:101990000F5F11E0AEC00130C1F5833739F4009319
:1019A000B8018EE991E00E94C21E02C01092B801F7
:1019B000182F10531F1539F08CE496E060E170E0A9
:1019C000412F0E948A2886E0891568F020E030E0E7
:1019D000992011F021E030E08091B80190E02817C3
:1019E000390709F408C18091B801882331F08CE4EB
:1019F00096E062E170E041E005C08CE496E062E1CF
:101A000070E040E00E948A28F6C0023069F4182F86
:101A100010531B1509F4F1C08CE496E061E170E00D
:101A2000412F0E948A28E9C0033069F4182F10530F
:101A30001A1509F4E4C08CE496E063E170E0412FEC
:101A40000E948A28DCC0043009F052C019821A8230
:101A50001B821C828093D80111E00EC08EE991E0B8
:101A60000E94C21E8D30E9F08A30D9F0E12FF0E0FB
:101A7000E852FE4F80831F5F2091B0013091B10189
:101A80004091B2015091B3018091A8019091A901B8
:101A9000A091AA01B091AB01281739074A075B074B
:101AA000E9F6E12FF0E0E852FE4F108288ED91E078
:101AB00060E070E040E150E00E94260169837A8393
:101AC0008B839C8380E090E0F301E80FF91FE081B5
:101AD000F999FECF1FBA449692BD81BDE0BD0FB605
:101AE000F894FA9AF99A0FBE43978430910561F7FA
:101AF00010E02091B0013091B1014091B2015091BC
:101B0000B3018091A8019091A901A091AA01B0917F
:101B1000AB01281739074A075B0709F02FCF8EE979
:101B200091E00E94891DA7FC0FC09A2D1092B90167
:101B3000A0FE03C081E08093B9011092070191FFDC
:101B400003C081E08093070109811A812B813C81C8
:101B50008F2D6B2D4A2D0E94710B85E08F1528F17A
:101B6000EF2DF0E0EE0FFF1FE05FFE4F00811181CF
:101B700088EF96E00E94AF2EFF20B9F081E08093BD
:101B800005018091B801882341F088EF96E040EC90
:101B900052E160E070E027E006C0A80160E070E07C
:101BA00088EF96E026E00E940B2E0E943C1583E011
:101BB0008B1538F1EB2DF0E0EE0FFF1FE05FFE4FCD
:101BC0002081318121153105E1F081E0809306010A
:101BD00040E050E0CA01B9019695879577956795E1
:101BE00060507C4D8B409F4F0E940E33CA01B9015B
:101BF0000E94491706C0F12E7BCFB12E79CFA12EBE
:101C000077CF0F900F900F900F90CF91DF911F9192
:101C10000F91FF90EF90DF90CF90BF90AF909F908B
:101C20007F906F90089585E593E00E940B1087ECFC
:101C300091E00E94FC1487EC91E00E942F1588230C
:101C400059F087EC91E060E00E94E61487EC91E0A7
:101C500060E00E94F11408955D980895DF92EF927C
:101C6000FF920F931F93DF93CF9300D0CDB7DEB7D2
:101C7000FE0131962DEF33E0AF014F5F5F4FF999D1
:101C8000FECF32BD21BDF89A80B580832F5F3F4FD4
:101C9000E417F50711F03196F2CF89819A810F97F9
:101CA000F9F08FE090E09A83898380E090E09E01D4
:101CB0002F5F3F4FF901E80FF91FE081F999FECF3F
:101CC0001FBA83509C4F92BD81BDE0BD0FB6F89402
:101CD000FA9AF99A0FBE8C5F93408230910551F7C2
:101CE0001092D6011092D70187E061E00E94A52BE7
:101CF00086E061E00E94A52B84E061E00E94A52BB4
:101D000085E061E00E94A52B8BB18F708BB982E0DA
:101D100061E00E94A52B5A9883E062E00E94A52B07
:101D20008AE061E00E94A52B5F9A64EF71E080E099
:101D300090E00E943D2B5C9A5A9A68EE73E080E036
:101D400090E00E943D2B5D9A0E94130E68EE73E0B6
:101D500080E090E00E943D2B8BB18F708BB95F9A31
:101D600010C05E9A5A9860E273E080E090E00E94B2
:101D70003D2B5E985A9A64EF71E080E090E00E94FB
:101D80003D2B82E691E06AE042E00E942D23882309
:101D900041F35A9A8BB18F708BB98BB18F708BB91D
:101DA0000E94F42A605D7A488F4F9F4F6093E5014F
:101DB0007093E6018093E7019093E801EE24FF24FD
:101DC0008701DD2417C00E941A08A0E0B0E0E80EE9
:101DD000F91E0A1F1B1FD3945F9A64EF71E080E025
:101DE00090E00E943D2B5F9864EF71E080E090E00E
:101DF0000E943D2B0E94F42A2091E5013091E601DA
:101E00004091E7015091E801621773078407950735
:101E1000D0F22D2D30E040E050E0C801B7010E9423
:101E20000E33285C30403093EA012093E9015F9A39
:101E30005C9A0E94F80B5D9A0E94130E64EF71E0A9
:101E400080E090E00E943D2B8BB18F708BB90F909A
:101E50000F90CF91DF911F910F91FF90EF90DF9046
:101E6000089581E0809354036093310310925203EC
:101E70001092530308952091300330E080912F0396
:101E8000281B3109C901089540912F038091300327
:101E9000481718F02FEF3FEF0AC0E42FF0E0E15FA2
:101EA000FC4F8081282F30E04F5F40932F03C90102
:101EB0000895E0912F0380913003E81718F0EFEFB9
:101EC000FFEF06C0F0E0E15FFC4F8081E82FF0E01B
:101ED000CF0108950895109258031092570388EE89
:101EE00093E0A0E0B0E08093590390935A03A0934D
:101EF0005B03B0935C0382E291E09093560380937E
:101F000055030895CF92DF92EF92FF920F931F93A4
:101F1000CF93DF937C016B018A0180915403882366
:101F2000A1F0C0E0D0E00DC0D701ED91FC91D60149
:101F3000AC0FBD1F0190F081E02DC7016C91099598
:101F40002196C017D10780F304C0CB01642F0E94F3
:101F5000B410C801DF91CF911F910F91FF90EF90C6
:101F6000DF90CF900895DF93CF930F92CDB7DEB778
:101F7000FC016983809154038823C9F08091530345
:101F8000803238F081E090E09383828320E030E07B
:101F900015C080915203E82FF0E0EE5CFC4F998170
:101FA00090838F5F809352038093530305C0CE01CB
:101FB000019661E00E94B41021E030E0C9010F9069
:101FC000CF91DF9108950F93062F8091310362E343
:101FD00073E04091530321E00E945F10109252037E
:101FE00010925303109254030F91089561E00E94E0
:101FF000E30F0895413208F040E2862F6FE073E06E
:102000000E94161010922F0380933003089521E050
:102010000E94FA0F089510922F031092300310922D
:102020005203109253030E9460120895382F4132D8
:1020300010F040E042C0809161038823E1F791E015
:1020400090936103209363038FEF8093CE031092EC
:102050008903415040938A034F5F909362038091BC
:102060006203330F832B809362038091640381307A
:1020700041F410926403809162038093BB0085EC6D
:1020800001C085EE8093BC00809161038130E1F353
:1020900080918903841710F44091890320E030E097
:1020A0000AC0FB01E20FF31FD901A759BC4F8C9165
:1020B00080832F5F3F4F2417A0F3842F08950F9341
:1020C0001F93582F122F413210F081E04AC08091A7
:1020D00061038823E1F782E0809361030093630347
:1020E0008FEF8093CE031092890340938A03A9E671
:1020F000B3E0FB0102C081918D938E2F861B841764
:10210000D0F31092620380916203550F852B809368
:10211000620380916403813041F4109264038091E2
:1021200062038093BB0085EC01C085EE8093BC0008
:10213000112321F0809161038230E1F38091CE037D
:102140008F3F11F480E00DC08091CE03803211F4F6
:1021500082E007C08091CE03803311F084E001C09B
:1021600083E01F910F910895482F613210F081E0B4
:10217000089580916103843011F082E008956093A6
:10218000AC03ABE8B3E0842F9C01F90102C081915C
:102190008D938E2F841B8617D0F380E008951F92B5
:1021A0000F920FB60F9211242F933F934F935F938B
:1021B0006F937F938F939F93AF93BF93EF93FF930F
:1021C0008091B90090E0887F90708036910509F485
:1021D000F2C081369105CCF58832910509F47BC0B7
:1021E00089329105B4F48031910509F46FC08131D1
:1021F00091053CF4009709F447C1089709F04FC1D5
:1022000065C08831910509F466C0809709F047C11F
:1022100082C08034910509F4A4C08134910544F44E
:102220008033910509F482C0C89709F038C189C08C
:102230008035910509F489C08835910509F496C067
:102240008834910509F02BC1AEC08839910509F495
:1022500013C189399105ECF48837910509F4ABC0B5
:10226000893791054CF48836910509F4A4C080376C
:10227000910509F014C19FC08838910509F4FCC08C
:102280008039910509F49DC08038910509F007C196
:1022900098C0803B910509F4C6C0813B91054CF480
:1022A000803A910509F49FC0883A910509F0F7C07A
:1022B000BAC0803C910509F4E3C0883C910509F45B
:1022C000DFC0883B910509F0EAC0C2C0809162037B
:1022D0008093BB00CFC09091890380918A039817A7
:1022E00068F490918903E92FF0E0E759FC4F808171
:1022F0008093BB009F5F90938903BCC08091630370
:10230000882309F44BC085ED8093BC008091BC000C
:1023100084FDFCCFC2C080E28093CE0385ED809324
:10232000BC008091BC0084FDFCCFB7C080E38093EB
:10233000CE0385ED8093BC008091BC0084FDFCCF72
:10234000ACC088E38093CE039BC0809189039091B9
:10235000BB00E82FF0E0E759FC4F90838F5F80933C
:1023600089039091890380918A0382C080918903B7
:102370009091BB00E82FF0E0E759FC4F90838F5F0E
:102380008093890380916303882341F085ED8093D6
:10239000BC008091BC0084FDFCCF7FC081E08093B5
:1023A000640384EA6EC085ED8093BC008091BC001C
:1023B00084FDFCCF72C083E0809361031092CD0353
:1023C00059C08091CD03803208F056C08091CD0372
:1023D0009091BB00E82FF0E0E355FC4F90838F5FB6
:1023E0008093CD0347C08091CD03803230F4E091DB
:1023F000CD03F0E0E355FC4F108285ED8093BC00E7
:102400008091BC0084FDFCCF109261036091CD03EC
:10241000E0916703F09168038DEA93E070E009951D
:102420001092CD032DC084E0809361031092AB0322
:102430001092AC03E0916503F091660309958091D9
:10244000AC03882329F481E08093AC0310928B03C2
:102450009091AB03E92FF0E0E557FC4F808180932A
:10246000BB009F5F9093AB039091AB038091AC0353
:10247000981710F485EC01C085E88093BC000FC06C
:1024800085EC8093BC0009C01092CE0385ED80934B
:10249000BC008091BC0084FDFCCF10926103FF91D1
:1024A000EF91BF91AF919F918F917F916F915F91CC
:1024B0004F913F912F910F900FBE0F901F90189545
:1024C0001092610381E0809363031092640382E1C0
:1024D00061E00E94E42B83E161E00E94E42BE9EBE0
:1024E000F0E080818E7F808380818D7F808388E48F
:1024F0008093B80085E48093BC000895EF92FF922A
:102500000F931F93CF93DF93582F162FE42E022F94
:10251000F32E85E593E0652F0E94310F85E593E06A
:10252000612F0E94B30F202F3F2DC901EC0110E055
:1025300006C085E593E069910E94B30F1F5F1E15E9
:10254000C0F385E593E00E94F60F90E0882309F43C
:1025500091E0892FDF91CF911F910F91FF90EF9024
:102560000895DF93CF930F92CDB7DEB7498341E053
:102570009E012F5F3F4F0E947E120F90CF91DF91FF
:1025800008952F923F924F925F926F927F928F9217
:102590009F92AF92BF92CF92DF92EF92FF920F93F2
:1025A0001F93DF93CF9300D000D00F92CDB7DEB74B
:1025B000882E6983942E3B832A830E94F42A5B0130
:1025C0006C01FF24EE24292C33242801662477246F
:1025D0004BC085E593E0682D0E94310F85E593E0BF
:1025E00069810E94B30F85E593E00E94F60F85E5AF
:1025F00093E0682D0E94310FA1014E19510941321B
:10260000510514F040E250E085E593E0682D0E940A
:1026100007102F2D332727FD30958A819B81280FA6
:10262000391F3D832C8385E593E00E943B0F892B66
:1026300009F452C00115110561F00E94F42A6A19CB
:102640007B098C099D09641575058605970508F0B9
:1026500043C085E593E00E94440FEC81FD818193A6
:10266000FD83EC83F394DFCFE91408F4B2CF0115B6
:102670001105C9F00E94F42A6A197B098C099D0989
:10268000980140E050E0621773078407950758F0FF
:102690002F2D332727FD3095892D90E028173907F6
:1026A00014F4FF24FA948F2D0F900F900F900F9039
:1026B0000F90CF91DF911F910F91FF90EF90DF90DE
:1026C000CF90BF90AF909F908F907F906F905F90D2
:1026D0004F903F902F90089585E593E00E94F60F6C
:1026E000892DF0E2F91508F480E2E80EBDCF0F93D2
:1026F0001F93FA01890141E09F010E94C1121F91BD
:102700000F910895DF92EF92FF920F931F93DF9343
:10271000CF930F92CDB7DEB7E82ED62EF42E122F20
:102720002091080130910901AE014F5F5F4F0E9477
:102730007713882341F1212F30E04F2D50E04F5F78
:102740005F4F421B530B81E090E002C0880F991F3E
:102750001A95E2F70197042E02C0880F991F0A9478
:10276000E2F7202F30E002C0220F331F4A95E2F734
:10277000482F4095598145238223482B49838E2D2C
:102780006D2D0E94B1120F90CF91DF911F910F918B
:10279000FF90EF90DF900895EF92FF920F931F93B9
:1027A000DF93CF930F92CDB7DEB7F82EE62E042F2E
:1027B000122F2091080130910901AE014F5F5F4F48
:1027C0000E9477132981112351F081E090E002C02B
:1027D000880F991F0A95E2F7422F482B0AC081E023
:1027E00090E002C0880F991F0A95E2F7482F4095A4
:1027F000422349838F2D6E2D0E94B1120F90CF91ED
:10280000DF911F910F91FF90EF900895CF92DF928B
:10281000EF92FF920F931F93DF93CF930F92CDB759
:10282000DEB7C42ED22E9701AE014F5F5F4F0E94DC
:102830007713682F882309F18D2D90E04C2D50E0FF
:102840004F5F5F4F481B590B21E030E002C0220F61
:10285000331FDA94E2F721503040042E02C0220FD9
:10286000331F0A94E2F78981822390E002C0959594
:1028700087954A95E2F7F8018083862F0F90CF91D4
:10288000DF911F910F91FF90EF90DF90CF9008950F
:10289000FC01608308958F929F92AF92BF92CF9276
:1028A000DF92EF92FF920F931F937C016B015A010D
:1028B00049019C012F5F3F4F0091080110910901D0
:1028C000FC01808163E446E00E94C112F70191811E
:1028D00080E0228130E0822B932BF601918380836C
:1028E000F701938180E0248130E0822B932BF50166
:1028F00091838083F701958180E0268130E0822BEF
:10290000932BF401918380831F910F91FF90EF909F
:10291000DF90CF90BF90AF909F908F9008958F924F
:102920009F92AF92BF92CF92DF92EF92FF920F935E
:102930001F937C016B015A0149019C012F5F3F4F9E
:102940000091080110910901FC0180816BE346E0D0
:102950000E94C112F701918180E0228130E0822B38
:10296000932BF60191838083F701938180E024818A
:1029700030E0822B932BF50191838083F7019581C1
:1029800080E0268130E0822B932BF40191838083B9
:102990001F910F91FF90EF90DF90CF90BF90AF907D
:1029A0009F908F900895FC01262F80816BE646E072
:1029B0000E94CC1308950F93FC01062F80816BE6D3
:1029C00042E023E00E9482130F9108950F93FC01CF
:1029D000062F80816CE144E022E00E9482130F9177
:1029E00008950F93FC01062F80816BE144E022E003
:1029F0000E9482130F9108950F931F938C0161E041
:102A00000E94DB14C80160E00E94F114C80160E07C
:102A10000E94E614C80160E00E94D3141F910F9138
:102A20000895CF92DF92EF92FF920F931F936C0164
:102A30008C010F5F1F4FE0900801F0900901FC012D
:102A4000808165E746E026E00E940614F601818158
:102A50001F910F91FF90EF90DF90CF9008950E940B
:102A6000111590E0843309F491E0892F0895809145
:102A70002A048823E1F7089580916F008B7F80936B
:102A80006F0080916F008F7D80936F008091CF03E6
:102A90008093D00380912A048823E1F780916F000E
:102AA0008D7F80936F000895282F90912D049F5F54
:102AB000983008F090E080912E048917E1F33FB739
:102AC000F89480912A04882341F0E92FF0E0E15D39
:102AD000FB4F208390932D041DC081E080932A0436
:102AE00020932B0410922C0482E086BB80916F000F
:102AF000826080936F00809180008F7380688093E4
:102B00008000809184009091850040969093890088
:102B1000809388003FBF0895862F0E94541581E05E
:102B200090E008951F920F920FB60F9211242F93E9
:102B30003F934F935F936F937F938F939F93EF9305
:102B4000FF9340912A0450912B04209188003091EA
:102B50008900609126047091270480912C041FC085
:102B6000260F371F952F917056954F5F9817B9F024
:102B7000992321F080918000806C04C080918000B6
:102B80008F73806880938000309389002093880041
:102B900090932C0450932B0440932A043BC049305B
:102BA000F8F2493039F48AE080932A048091800059
:102BB000806C28C080912D04E0912E048E1769F45A
:102BC00010922A04809180008F73809380008091FE
:102BD0006F008D7F80936F001DC081E080932A0479
:102BE000EF5FE83008F0E0E0E0932E04F0E0E15D14
:102BF000FB4F808180932B0410922C0480918000E5
:102C00008F73806880938000260F371F3093890070
:102C100020938800FF91EF919F918F917F916F9109
:102C20005F914F913F912F910F900FBE0F901F908A
:102C300018951F920F920FB60F9211241F932F9386
:102C40003F934F935F936F937F938F939F93AF9334
:102C5000BF93EF93FF93209186003091870090916E
:102C60002204992341F0809181008F7B8093810021
:102C70001092220408C080918100806480938100BA
:102C800080E88093220470912104772331F5992301
:102C900009F06CC08091240490912504820F931F49
:102CA00090938B0080938A0084E086BB80916F00B4
:102CB000846080936F008091260490912704280FF0
:102CC000391F96958795280F391F30932904209333
:102CD000280481E08093210449C040912804509148
:102CE000290410912204E0912604F09127046091B8
:102CF0002304AA27BB27AE1BBF0BC901841B950B5E
:102D000097FD2CC06695612B7F5F8A0F9B1F7930E2
:102D100018F44E0F5F1FF4CF6093230480916F006F
:102D20008B7F80936F009091D0039F5F903508F068
:102D300090E08091CF03981739F0E92FF0E0EF523F
:102D4000FC4F60839093D003809181008F7B8093B0
:102D50008100109222041092210408C06093230481
:102D6000509329044093280470932104FF91EF911C
:102D7000BF91AF919F918F917F916F915F914F9193
:102D80003F912F911F910F900FBE0F901F9018959C
:102D90001F920F920FB60F9211242F938F939F9330
:102DA000EF93FF9380916F008B7F80936F008091F2
:102DB00081008F7B80938100909121048091220477
:102DC00080582091230403C02695282B9F5F9930BB
:102DD000D8F3209323049091D0039F5F903508F09F
:102DE00090E08091CF03981739F0E92FF0E0EF528F
:102DF000FC4F20839093D003109221048091810096
:102E00008F7B8093810010922204FF91EF919F911C
:102E10008F912F910F900FBE0F901F90189580915A
:102E2000D003E091CF038E1719F42FEF3FEF0EC0C0
:102E30002E2F2F5F203508F020E0E22FF0E0EF5238
:102E4000FC4F80812093CF03282F30E0C9010895E3
:102E50008091D003E091CF038E1719F4EFEFFFEFCD
:102E600006C0F0E0EF52FC4F8081E82FF0E0CF0188
:102E700008959091D0038091CF03292F30E0482FFF
:102E800050E0981710F4205B3F4F241B350BC9010D
:102E900008959B01AC012D3A8BE1380780E048078B
:102EA00080E0580730F410926F001092800081E8A3
:102EB00014C063E056954795379527956A95D1F7E5
:102EC0002D3A8BE1380780E0480780E05807D0F5BD
:102ED00010926F001092800082E8809381003093FE
:102EE000270420932604CA01B90125E230E040E01E
:102EF00050E00E94C83252E0969587957795679585
:102F00005A95D1F7709325046093240488E062E019
:102F10000E94A52B89E061E00E94E42B89E061E03A
:102F20000E94A52B109221041092D0031092CF037F
:102F300010922A0410922D0410922E0480E286BB77
:102F400080936F0008958091C10085FDFCCF809132
:102F5000C00085FFF8CF6093C60081E090E008953F
:102F600010923A041092390482E491E0909338046C
:102F7000809337040895FF920F931F93CF93DF93AD
:102F80008B010E94F42AEB01FF24FA9409C00E94ED
:102F9000F42A6C1B7D0B6017710710F080E008C0ED
:102FA000FEBC0DB407FEFDCF8EB58F3F81F781E0EB
:102FB000DF91CF911F910F91FF900895FC018081C7
:102FC00061E00E94E42B8FEF8EBD0DB407FEFDCFB4
:102FD0000895CF93DF93EC01DA016EBD0DB407FEC7
:102FE000FDCF8C918EBD1196EC91119782E090E00F
:102FF0000DB407FEFDCFEEBD22E08030920731F028
:10300000FD01E80FF91FE0810196F2CF0DB407FE34
:10301000FDCF8FEF8EBD0DB407FEFDCF8FEF8EBDC0
:103020000DB407FEFDCF8FEF8EBD0DB407FEFDCFB3
:103030008EB58B838F71853011F481E006C083E1FA
:103040008983CE010E94DE1780E0DF91CF91089541
:10305000BF92CF92DF92EF92FF920F931F93CF9385
:10306000DF93EC016B017A010E94F42A8B01BB24EF
:10307000BA9409C00E94F42A601B710B6D52714012
:1030800010F081E10BC0BEBC0DB407FEFDCF8EB5C4
:103090008B838F3F79F38E3F39F08FE08983CE01A8
:1030A0000E94DE1780E030C0D7011197EF28D9F0D9
:1030B0008FEF8EBD20E030E09FEF0BC00DB407FE18
:1030C000FDCF8EB59EBDF601E20FF31F80832F5F0B
:1030D0003F4F2A173B0790F30DB407FEFDCF8EB587
:1030E000AC0DBD1D8C931B828FEF8EBD0DB407FE02
:1030F000FDCF8EB58FEF8EBD0DB407FEFDCF8EB523
:10310000CE010E94DE1781E0DF91CF911F910F91D8
:10311000FF90EF90DF90CF90BF9008950F931F9393
:103120008C018BE394E0F80162810E947223F80124
:10313000808160E00E94E42B1F910F910895FF921F
:103140000F931F93DF93CF9300D000D0CDB7DEB79E
:103150008C01F62E29833A834B835C830E948E1860
:10316000C80168E572E00E94BB178F2D80648EBD98
:103170000DB407FEFDCFFE0131969E012350304075
:1031800083818EBD0DB407FEFDCF3197E217F307A3
:10319000B9F7FF2011F087E801C085E98EBD0DB4B5
:1031A00007FEFDCF8CE0F81631F48FEF8EBD0DB425
:1031B00007FEFDCF8EB590E02FEF2EBD0DB407FEBC
:1031C000FDCF8EB587FF02C09150B9F7F801838318
:1031D0000F900F900F900F90CF91DF911F910F9153
:1031E000FF900895CF92DF92EF92FF920F931F937B
:1031F000CF93DF93EC017A018B0169018C818330DD
:1032000039F099E0EE0CFF1C001F111F9A95D1F7C1
:10321000CE0168E1A80197010E949F18882319F048
:1032200086E089830CC0CE016EEFA6010E94E917EB
:10323000882329F0CE010E94DE1781E004C0CE0170
:103240000E94DE1780E0DF91CF911F910F91FF90D8
:10325000EF90DF90CF900895CF92DF92EF92FF92A0
:103260000F931F93CF93DF93EC017A018B016901D8
:103270008C81833039F0B9E0EE0CFF1C001F111F68
:10328000BA95D1F7CE0161E1A80197010E949F187C
:10329000882339F084E08983CE010E94DE1780E024
:1032A00006C0CE01B60140E052E00E942818DF912E
:1032B000CF911F910F91FF90EF90DF90CF900895E5
:1032C000BF92CF92DF92EF92FF920F931F93CF9313
:1032D000DF93EC01B42E1C82198268830E94F42AC9
:1032E0006B01888161E00E94A52B888161E00E94CA
:1032F000E42B8BE394E00E948C2380E48A838BE3AD
:1033000094E060E40E94722380E09FEF9EBD0DB4C4
:1033100007FEFDCF8F5F8A30C9F709C00E94F42AEB
:103320006C197D09615D774010F081E063C0CE01CA
:1033300060E020E030E040E050E00E949F188130E3
:1033400069F71FEFCE0168E02AEA31E040E050E083
:103350000E949F18853011F481E00DC080E01EBDF1
:103360000DB407FEFDCF9EB58F5F8430C1F79B8300
:103370009A3A31F482E08C838C81823051F40DC012
:103380000E94F42A6C197D09615D7740D8F282E0D1
:1033900031C0EE24FF2487010FC0E12CF12C012D58
:1033A00080E4182F09C00E94F42A6C197D09615D20
:1033B000774010F08AE01EC0CE0167E320E030E0E5
:1033C00040E050E00E949F18CE0169E2A8019701F9
:1033D0000E949F18882339F78C81823031F5CE0105
:1033E0006AE320E030E040E050E00E949F1888232C
:1033F00039F088E08983CE010E94DE1780E01AC090
:103400008FEF8EBD0DB407FEFDCF8EB5807C803C66
:1034100011F483E08C8380E09FEF9EBD0DB407FE26
:10342000FDCF2EB58F5F8330C1F7CE010E94DE172E
:10343000BA8281E0DF91CF911F910F91FF90EF90C1
:10344000DF90CF90BF9008950F931F93CF93DF939A
:10345000DC01EB018A0180E090E020E2FE01E80F50
:10346000F91F208301968B309105C1F757E040E0AA
:1034700024C0622F2E3219F084E891E007C05A3040
:1034800051F15AE048E018C0321729F1FC010196C9
:1034900034913323C9F75417F0F02132E0F02F377D
:1034A000D0F4822F81568A3110F4622F6052FE01CF
:1034B000E40FF11D60834F5F11962C91222311F0D0
:1034C0002F32B9F6F801B183A08390E08881803271
:1034D00019F091E001C090E0892FDF91CF911F9109
:1034E0000F910895CF92DF92EF92FF920F931F9367
:1034F000DF93CF9300D000D0CDB7DEB77C01FC01C5
:1035000086899789A08DB18D89839A83AB83BC838B
:1035100000E010E06E010894C11CD11C49815A8161
:103520006B817C81D70114968D919C9115979601A2
:103530000E949C26882379F1D7011496ED91FC9185
:1035400015978481080F111DB0E100301B0718F595
:1035500029813A814B815C818289803131F4285FF5
:103560003F4F40405040D0F205C0285F3F4F4F4F83
:103570005F40A0F2C801A0E0B0E029E0880F991FE9
:10358000AA1FBB1F2A95D1F7F701828B938BA48BBF
:10359000B58B81E001C080E00F900F900F900F90ED
:1035A000CF91DF911F910F91FF90EF90DF90CF901F
:1035B0000895CF93DF93EC01FB018A818823D1F535
:1035C0007D836C8382898031C9F582E08A831E8A7B
:1035D0001F8A188E198E83899489A0E0B0E035E0A7
:1035E000880F991FAA1FBB1F3A95D1F78A8B9B8B17
:1035F000AC8BBD8B0FC083E08A8385899689A789B0
:10360000B08D8E8B9F8BA88FB98FCE010E94721ABE
:10361000882381F081E089831E821F8218861986A3
:103620001A861B861C861D861E861F86188A198A86
:103630001B8201C080E0DF91CF9108958032D1F7E5
:10364000DACF6F927F928F929F92AF92BF92CF927A
:10365000DF92EF92FF920F931F93CF93DF93EC01D2
:103660007A018B012A81222309F480C08A899B89EF
:10367000AC89BD8984179507A607B70708F476C0FB
:1036800085C0E114F1040105110551F41E821F8269
:10369000188619861A861B861C861D8681E067C0DF
:1036A0002A853B854C855D85EC81FD81818590E097
:1036B0000996215030404040504039014A01082EBF
:1036C00004C096948794779467940A94D2F72F5FF6
:1036D0003F4F4F4F5F4F0894E108F108010911096E
:1036E0005701680104C0D694C794B794A7948A95EB
:1036F000D2F70894E11CF11C011D111DA614B7049A
:10370000C804D90428F0211531054105510549F4B3
:103710008E899F89A88DB98D8E839F83A887B9874D
:1037200016C0A618B708C808D90811C04E815F8115
:10373000688579858C819D8194010E949C260894DE
:10374000A108B108C108D108882331F40FC046E0B0
:10375000842E912C8C0E9D1EA114B104C104D104A1
:1037600029F7EA86FB860C871D8798CF80E0DF91DA
:10377000CF911F910F91FF90EF90DF90CF90BF906E
:10378000AF909F908F907F906F900895223009F0B6
:1037900078CFE7CFCF93DF93EC01462F6E857F85FF
:1037A000888999890E941824AC01009719F420E0B7
:1037B00030E00AC08B81282F30E065E0220F331FF4
:1037C0006A95E1F7240F351FC901DF91CF91089564
:1037D0000F931F93CF93DF938C01FC018281882389
:1037E000F1F1818187FF38C0C80161E00E94CA1BE6
:1037F000EC010097A1F18881853E89F1F801828171
:10380000823040F482899389A489B5898C8F9D8FF9
:10381000AE8FBF8FF801868997899B8F8A8F8689A3
:103820009789A08DB18DCD01AA27BB279D8B8C8B4D
:10383000E0913E04F0913F04309751F0BE016A5E82
:103840007F4FCE0148960995888D998D9B8B8A8BE9
:10385000F80181818F7781830E94D02304C081E0A9
:10386000F801808380E0DF91CF911F910F9108953F
:103870006F927F928F929F92AF92BF92CF92DF9280
:10388000EF92FF920F931F93DF93CF9300D000D05E
:10389000CDB7DEB77C015A016B01DC0112968C9129
:1038A0001297813009F091C011968C9181FF8DC0E3
:1038B000A0C00097A105B10511F481E087C0F70110
:1038C0006284738484849584C701B601A5010E9433
:1038D000211B882309F479C0D70114968D919C91FE
:1038E0001597A114B104C104D10489F456964D91E1
:1038F0005D916D917C9159970E940B27882309F463
:1039000064C0F701168A178A108E118E44C0D70141
:1039100016964D915D916D917C9119979E012F5F47
:103920003F4F0E949C26882309F44FC0D70114966C
:10393000ED91FC91159749815A816B817C81828937
:10394000803149F4483FBFEF5B07B0E06B07B0E060
:103950007B0748F020C0483F8FEF58078FEF68077C
:103960008FE07807C0F4CF010E940B27882369F10C
:10397000D70116964D915D916D917C911997149692
:103980008D919C9115970FEF1FEF2FEF3FE00E9455
:103990002C268823D1F0F701A28AB38AC48AD58A5B
:1039A000818180688183C7010E94E81B882369F0B8
:1039B000B601A5016A147B048C049D0410F4B401C3
:1039C000A301C7010E94211B01C080E00F900F904E
:1039D0000F900F90CF91DF911F910F91FF90EF907B
:1039E000DF90CF90BF90AF909F908F907F906F901F
:1039F0000895F70182899389A489B5898417950769
:103A0000A607B70708F055CFE0CF1F93CF93DF93FA
:103A1000EC01142F262F30E0F90185E0EE0FFF1F97
:103A20008A95E1F7EB5BFB4F8385817121F0842F51
:103A3000827109F064C08091450690914606A0917C
:103A40004706B09148068E879F87A88BB98B6B83FA
:103A5000F901B5E0EE0FFF1FBA95E1F7EB5BFB4F05
:103A60002489358940E050E0A901332722272E8B95
:103A70003F8B488F598F828D938DA0E0B0E0282B2B
:103A8000392B4A2B5B2B2E8B3F8B488F598F83858D
:103A900090E088719070009751F4848D958DA68D7B
:103AA000B78D8A8B9B8BAC8BBD8B81E008C0409718
:103AB00031F5CE010E94721A882309F184E08A83CD
:103AC000812F8F7089831E821F82188619861A861D
:103AD0001B861C861D8614FF18C0CE0140E050E0F6
:103AE00060E070E00E94381C882379F408C04A899D
:103AF0005B896C897D89CE010E94211B02C01A82DC
:103B000080E0DF91CF911F91089515FDF0CF81E006
:103B1000F8CF0F931F938C010E94E81BF8011282CB
:103B20001F910F910895CF93DF93EC0140E050E097
:103B300060E070E00E94381C882369F0CE0161E0EB
:103B40000E94CA1BFC01009731F085EE80831A8227
:103B50000E94D02301C080E0DF91CF9108952F9281
:103B60003F924F925F926F927F928F929F92AF920D
:103B7000BF92CF92DF92EF92FF920F931F93DF934A
:103B8000CF9300D0CDB7DEB74C011A01DC011296FD
:103B90008C911297882309F4B4C011968C9180FF00
:103BA000B0C0C7C015012E183F082B01F40136968E
:103BB000FA83E98331019FC0D4011A962D913D917A
:103BC0004D915C911D979FEFA92E91E0B92EA222F5
:103BD000B3221496ED91FC91159779018A0189E041
:103BE00016950795F794E7948A95D1F794811296E4
:103BF0008C91823049F4458956896789708D4E0DC4
:103C00005F1D601F711F35C0D92EDA94DE20A1140C
:103C1000B10401F5DD20F1F421153105410551050F
:103C200051F4F40186899789A08DB18D868397839D
:103C3000A087B1870FC0D40116964D915D916D910B
:103C40007C911997CF0129813A810E949C26882373
:103C500009F457C0F40146815781608571858481DC
:103C600095810E94B023AB01BC014D0D511D611D1A
:103C7000711DA114B10499F4F0E06F16F2E07F0613
:103C800070F08091450690914606A0914706B0914C
:103C90004806481759076A077B0709F067C0CB0138
:103CA000BA0140E00E941824009759F140E052E028
:103CB0004A195B0983014615570508F48A019C01DE
:103CC0002A0D3B1DC201B901A8010E943802400E15
:103CD000511E980140E050E0F40182859385A4854F
:103CE000B585820F931FA41FB51F82879387A48772
:103CF000B587601A710A6114710409F05DCFA101E2
:103D000002C04FEF5FEFCA010F900F90CF91DF918C
:103D10001F910F91FF90EF90DF90CF90BF90AF90E9
:103D20009F908F907F906F905F904F903F902F90DB
:103D30000895D4015296AD90BD90CD90DC905597EA
:103D40001A96ED90FD900D911C911D979A0140E0FF
:103D500050E0D601C5018E199F09A00BB10B2817A1
:103D600039074A075B0708F01DCF1FCF80914A062D
:103D700090914B0692010E942C19882311F200E0C9
:103D800012E0A5CFDF93CF930F92CDB7DEB7BE0180
:103D90006F5F7F4F41E050E00E94AF1D019719F027
:103DA0002FEF3FEF03C08981282F30E0C9010F902A
:103DB000CF91DF910895CF93DF93EC019C012A5FAF
:103DC0003F4F8C819D8141E050E060E070E00E94B7
:103DD00072278823A1F08E899F89A88DB98D0097BD
:103DE000A105B10559F48E819F81A885B9858E8B77
:103DF0009F8BA88FB98F89818068898381E0DF914B
:103E0000CF9108952F923F924F925F926F927F923F
:103E10009F92AF92BF92CF92DF92EF92FF920F9359
:103E20001F93DF93CF9300D000D0CDB7DEB76C01E6
:103E3000162F072F1A01DC0112968C9112978130F0
:103E400009F046C111968C9181FF42C15DC1F60116
:103E5000428953896489758982859385A485B5854E
:103E600084179507A607B70731F0C6010E94211BEA
:103E7000882309F42DC1812F902F9C012901310144
:103E8000EDC0D6011496ED91FC911597DA01C901A8
:103E900019E0B695A795979587951A95D1F79480CF
:103EA0009A949822AFEFAA2EA1E0BA2EA222B322B2
:103EB000992009F052C0A114B10409F04EC0D601F6
:103EC00016964D915D916D917C9119974115510513
:103ED0006105710571F1CF019E012F5F3F4F0E9477
:103EE0009C26882309F4F4C029813A814B815C81A6
:103EF000D6011496ED91FC9115978289803149F491
:103F0000283FBFEF3B07B0E04B07B0E05B0748F04E
:103F100019C0283FEFEF3E07EFEF4E07EFE05E07D7
:103F200088F4D60116962D933D934D935C93199783
:103F300014C0F60186899789A08DB18D0097A105DF
:103F4000B10531F4C6010E94DB1E882331F4C0C0E4
:103F5000F60186839783A087B187D60116964D9187
:103F60005D916D917C91199714968D919C91159707
:103F70000E94B0237B018C01E90CF11C011D111D75
:103F8000A114B104A9F4B0E06B16B2E07B06A8F569
:103F9000F601228533854485558582899389A489D4
:103FA000B589281739074A075B0710F045E001C0BB
:103FB00041E0C801B7010E941824009709F488C0A5
:103FC00040E052E04A195B0983014615570508F4A1
:103FD0008A019C012A0D3B1DC901B201A8010E9462
:103FE0003802A00EB11EF0E0AF16F2E0BF0611F5E8
:103FF0000E9415248823F1F46BC0809145069091AE
:104000004606A0914706B09148068E159F05A00769
:10401000B10711F40E94A12380914A0690914B06AA
:10402000B801A70192010E94F218882309F450C038
:1040300000E012E0980140E050E0F60182859385AF
:10404000A485B585820F931FA41FB51F8287938710
:10405000A487B587400E511E601A710AD6011A96C0
:104060002D913D914D915C911D976114710409F062
:1040700008CF52968D919D910D90BC91A02D8217E5
:104080009307A407B50748F4F601228B338B448BC2
:10409000558B81818068818310C080913E0490910E
:1040A0003F04892B51F02114310439F0D6011196C7
:1040B0008C911197806811968C93F601818183FF12
:1040C00005C0C6010E94E81B882311F0A10105C0AC
:1040D00081E0D6018C934FEF5FEFCA010F900F90F4
:1040E0000F900F90CF91DF911F910F91FF90EF9064
:1040F000DF90CF90BF90AF909F907F906F905F9038
:104100004F903F902F90089582FDA1CEB4CE9F9204
:10411000AF92BF92CF92DF92EF92FF920F931F93D5
:10412000CF93DF938C01FC0182899389A489B5899F
:10413000805E9F4FAF41B04008F05CC0C8010E9454
:10414000DB1E882309F456C0D80116964D915D9167
:104150006D917C91199714968D919C9115970E9461
:10416000B0235B016C0145E00E941824EC0100972C
:1041700009F442C080E092E0FE019C0111922150BE
:104180003040E1F79C2EED2EFF24F39411C0B601D0
:10419000A5014F0D511D611D711D80914A06909121
:1041A0004B06292D3E2D0E94F218882319F1F39415
:1041B000D8011496ED91FC9115972481F21638F3ED
:1041C00030E040E050E089E0220F331F441F551FCC
:1041D0008A95D1F752968D919D910D90BC91A02D0D
:1041E000820F931FA41FB51FF801828B938BA48BA2
:1041F000B58B02C0C0E0D0E0CE01DF91CF911F911E
:104200000F91FF90EF90DF90CF90BF90AF909F9075
:1042100008953F924F925F926F927F928F929F92FA
:10422000AF92BF92CF92DF92EF92FF920F931F93C4
:10423000CF93DF934C01EB01442E352E522E8C810F
:104240009D81F40195838483CB0140E050E060E0E0
:1042500070E00E94211B77244FC0CE010E94C21E35
:1042600097FDABC08A859B85AC85BD8581509E4FEF
:10427000AF4FBF4F8A879B87AC87BD87A09045060D
:10428000B0904606C0904706D090480625E4E22E3E
:1042900024E0F22E00E010E0602EF70180818823F8
:1042A00011F0853E79F4772041F4F401A686B786B3
:1042B000C08AD18A638277247394F701808188232E
:1042C00091F428C0B80195E0660F771F9A95E1F741
:1042D0006B5B7B4F842D932D4BE050E00E942B02B3
:1042E000009709F47DC00F5F1F4F80E290E0E80E59
:1042F000F91E0031110581F62A853B854C855D85C7
:104300008A899B89AC89BD89281739074A075B07C9
:1043100008F4A3CF56FE51C051FE4FC0772051F094
:10432000F4016380C40161E00E94CA1BEC010097A4
:1043300061F443C08A81823009F43FC0CE010E94FB
:1043400087200097D1F1EC01662480E2FE011192F2
:104350008A95E9F7DE01242D332DC901FC018BE09C
:1043600001900D928150E1F7E0913E04F0913F04FD
:10437000309739F0BE01625F7F4FCE0140960995BC
:1043800008C081E298E2998B888B80E098E09F8753
:104390008E87888999899B8B8A8B998F888F8E8548
:1043A0009F859F8B8E8B0E94D023882331F0C40180
:1043B000662D452D0E94051D01C080E0DF91CF9143
:1043C0001F910F91FF90EF90DF90CF90BF90AF9033
:1043D0009F908F907F906F905F904F903F90089547
:1043E00057FEE5CFEACF2F923F924F925F926F92A6
:1043F0007F928F929F92AF92BF92CF92DF92EF9275
:10440000FF920F931F93DF93CF93CDB7DEB7C454C2
:10441000D0400FB6F894DEBF0FBECDBF3C016B019C
:10442000DE01A05CBF4F11965C934E9323962FAF95
:1044300023976115710509F483C01E8618A6FC0137
:104440008281882309F07CC01C861EA2FA0180812B
:104450008F32F1F086015CE0E52EF12CEC0EFD1EB2
:1044600040E4A42EB12CAC0EBD1E4E010894811C5C
:10447000911C2596FFAEEEAE259736E2232E312C09
:104480002C0E3D1E270124C01196B183A08301C0CC
:10449000FD01A081B1818C918F32B1F3D6011296CA
:1044A0008C91129782508230A8F28E010A5D1F4FC4
:1044B00014966D917C911597C8010E94D91A882392
:1044C00051F63EC0342D252D8701832F922F7C017C
:1044D000F50180819181B401A5010E94241A8823ED
:1044E00029F42EC03196D501ED93FC93D501ED91C1
:1044F000FC9180818F32B1F38823C9F0C701B801E4
:10450000A40121E00E9409218823D1F00C151D058A
:1045100019F0C8010E94891D2596EEADFFAD2597C3
:10452000EE16FF0679F6C101322D292FCDCFC3013A
:10453000B801A40123962FAD23970E94092101C041
:1045400080E0CC5BDF4F0FB6F894DEBF0FBECDBF6F
:10455000CF91DF911F910F91FF90EF90DF90CF905F
:10456000BF90AF909F908F907F906F905F904F9093
:104570003F902F9008950F931F93DF93CF93CDB764
:10458000DEB76A970FB6F894DEBF0FBECDBF9C01B1
:10459000AB0119821B828E010F5F1F4FC801B90149
:1045A00022E00E94F321882319F0C8010E94931D84
:1045B0006A960FB6F894DEBF0FBECDBFCF91DF91E4
:1045C0001F910F910895FB01242F60913C0470917D
:1045D0003D04AF010E94F3210895DF93CF93CDB73F
:1045E000DEB76A970FB6F894DEBF0FBECDBF9C0151
:1045F000AB0119821B82CE010196B90121E00E9414
:10460000F3216A960FB6F894DEBF0FBECDBFCF91EF
:10461000DF9108954E960E94BB2208954E960E9407
:10462000ED220895CF93DF93EC01662331F06E966F
:10463000D0933D04C0933C046E9788A1882321F059
:10464000CE014E960E94891DCE014E962596BE0142
:104650000E94D91ADF91CF9108950F931F93CF93A2
:10466000DF93EC010E9460198823C9F08E010B5F73
:104670001F4FC801BE0141E00E945C24882339F429
:10468000C801BE0140E00E945C24882341F0CE01B5
:1046900061E00E941223882319F081E001C080E0CC
:1046A000DF91CF911F910F910895DF93CF930F92D8
:1046B000CDB7DEB769830496BE016F5F7F4F41E0DF
:1046C00050E00E94021F20E030E0019711F421E049
:1046D00030E0C9010F90CF91DF91089504960E94B8
:1046E000021F089540E082E002C0880F4F5F8617E6
:1046F00010F44630D1F7242F30E0C9019595879505
:1047000080658CBD40FF02C080E004C080E0463080
:1047100009F081E08DBD08958AE061E00E94E42BFC
:104720008AE061E00E94A52B8CE060E00E94A52B4E
:104730008BE061E00E94A52B8DE061E00E94A52B3B
:1047400008958FEF9FEFAFEFBFEF809345069093F3
:104750004606A0934706B09348061092490608956E
:104760000F931F938C01CB01BA01625070408040BF
:104770009040F801248130E040E050E00E94C832CF
:104780009B01AC01F80182859385A485B585280F2E
:10479000391F4A1F5B1FB901CA011F910F9108956C
:1047A0008091490680FF3DC04091450650914606E4
:1047B000609147067091480680914A0690914B0699
:1047C00025E434E00E94F218882369F180914906BB
:1047D00081FF22C0809140048230F0F0409141047A
:1047E00050914204609143047091440480914506C5
:1047F00090914606A0914706B0914806480F591F70
:104800006A1F7B1F80914A0690914B0625E434E095
:104810000E94F218882339F0809149068E7F809398
:10482000490681E0089580E008950E94D02308950C
:10483000DF92EF92FF920F931F937B018C01D42E96
:104840008091450690914606A0914706B091480692
:104850008E159F05A007B107E1F00E94D0238823A1
:1048600011F1D2FC0CC080914A0690914B06B80120
:10487000A70125E434E00E942C198823A1F01092AE
:104880004906E0924506F0924606009347061093CB
:10489000480683E0D822809149068D2980934906F5
:1048A00025E434E002C020E030E0C9011F910F91FF
:1048B000FF90EF90DF9008956F927F928F929F927A
:1048C000AF92BF92CF92DF92EF92FF920F931F931E
:1048D000CF93DF93EC01142F70934B0660934A063D
:1048E0001A8A82E090E0A0E0B0E088839983AA83EE
:1048F000BB83109249068FEF9FEFAFEFBFEF80931E
:10490000450690934606A0934706B0934806442375
:1049100021F466247724430136C0453008F0EFC007
:1049200060E070E080E090E040E00E941824DC014C
:10493000009709F4E4C0412F50E041505040FA0183
:1049400074E0EE0FFF1F7A95E1F7E80FF91FE254CC
:10495000FE4F808190E08F779070892B09F0CFC057
:1049600064E0440F551F6A95E1F7A40FB51FAA53E1
:10497000BE4F6D907D908D909C9061147104810468
:10498000910409F4BCC0C401B30140E00E941824A2
:104990005C01009709F4B3C0FC01838594858050C5
:1049A000924009F0ACC0F5012089222309F4A7C088
:1049B000468557854115510509F4A1C0209340044F
:1049C00085858C83198691E060E070E00AC0990FBC
:1049D0006F5F7F4F6830710509F491C089858F5FE3
:1049E00089878C81891799F7F5016689778961151F
:1049F000710519F080E090E005C0F50164A175A192
:104A000086A197A16093410470934204809343046C
:104A1000909344046A01EE24FF24C60CD71CE81CC2
:104A2000F91CCE86DF86E88AF98AF50101891289A8
:104A30001C8B0B8B30E040E050E00E94C8326C0DC4
:104A40007D1D8E1D9F1D6D8B7E8B8F8B988F35E00E
:104A5000000F111F3A95E1F701501E4F012F11274A
:104A60000695980140E050E0260F371F481F591F58
:104A70002A873B874C875D87F50183899489009756
:104A800021F07C0100E010E005C0F501E0A0F1A0FC
:104A900002A113A1C401B301621B730B840B950B1C
:104AA0006E0D7F1D801F911F098404C09695879508
:104AB000779567950A94D2F76D837E838F83988765
:104AC000653FFFE07F07F0E08F07F0E09F0718F4F5
:104AD0008CE08A8B14C0655F7F4F8040904010F45B
:104AE00080E10AC0F50184A595A5A6A5B7A58D8B83
:104AF0009E8BAF8BB88F80E28A8B81E001C080E013
:104B0000DF91CF911F910F91FF90EF90DF90CF90A9
:104B1000BF90AF909F908F907F906F90089542606C
:104B20000E94182408956F927F928F929F92AF9265
:104B3000BF92CF92DF92EF92FF920F931F93CF938A
:104B4000DF93EC018D819E81AF81B8852A89203168
:104B500019F0203209F06BC0E2E0EE2EF12C012DAD
:104B6000112DE80EF91E0A1F1B1F6E847F84888892
:104B70009988AA24BB24650151C0C401B30140E057
:104B80000E948F259C01009709F451C06A89603109
:104B900019F040E850E002C040E051E0CA01A0E056
:104BA000B0E0E816F9060A071B0708F4A701603110
:104BB00099F4F90120E030E080819181892B29F47A
:104BC0000894A11CB11CC11CD11C2F5F3F4F329611
:104BD0002417350788F316C0F90120E030E0808102
:104BE0009181A281B3810097A105B10529F40894B0
:104BF000A11CB11CC11CD11C2F5F3F4F3496241740
:104C0000350768F30894611C711C811C911CCA0152
:104C1000A0E0B0E0E81AF90A0A0B1B0BE114F1045A
:104C20000105110509F0A9CFA601950104C02FEFD8
:104C30003FEF4FEF5FEFB901CA01DF91CF911F91B5
:104C40000F91FF90EF90DF90CF90BF90AF909F902B
:104C50008F907F906F9008958F929F92AF92BF92A6
:104C6000CF92DF92EF92FF920F931F93CF93DF9338
:104C7000EC016A017B01480159014230510561058F
:104C8000710508F44BC08D819E81AF81B885019676
:104C9000A11DB11D84179507A607B70708F43EC0EC
:104CA0008A89803129F4252F362F472F55270BC0AD
:104CB0008032A1F59A01AB0117E0569547953795DB
:104CC00027951A95D1F78E859F85A889B989280FD0
:104CD000391F4A1F5B1FCA01B90141E00E948F259D
:104CE0009C010097D9F08A89803149F4F601F0706F
:104CF000EE0FFF1FE20FF31F918280820DC0F601BD
:104D0000EF77F070EE0FFF1FEE0FFF1FE20FF31FA4
:104D100080829182A282B38281E001C080E0DF9133
:104D2000CF911F910F91FF90EF90DF90CF90BF90A8
:104D3000AF909F908F900895CF92DF92EF92FF9265
:104D40000F931F93CF93DF93EC017A018B016901DD
:104D5000423051056105710508F453C08D819E8173
:104D6000AF81B8850196A11DB11D84179507A607CF
:104D7000B70708F446C08A89803129F45527412FA6
:104D8000302F2F2D0BC08032E1F59A01AB0167E087
:104D900056954795379527956A95D1F78E859F85C6
:104DA000A889B989280F391F4A1F5B1FCA01B90199
:104DB00040E00E948F259C01009719F18A8980317B
:104DC00059F4F701F070EE0FFF1FE20FF31F80811F
:104DD0009181A0E0B0E00EC0F701EF77F070EE0F28
:104DE000FF1FEE0FFF1FE20FF31F80819181A28151
:104DF000B381BF70F60180839183A283B38381E086
:104E000001C080E0DF91CF911F910F91FF90EF9053
:104E1000DF90CF9008958F929F92AF92BF92CF92E2
:104E2000DF92EF92FF920F931F93DF93CF9300D007
:104E300000D0CDB7DEB75C016A017B014E0108945A
:104E4000811C911CC501B701A60194010E949C26FA
:104E50008823B1F1C501B701A60100E010E020E010
:104E600030E00E942C26882359F1F5018081918140
:104E7000A281B381C816D906EA06FB0620F4C082D7
:104E8000D182E282F382C980DA80EB80FC80F50176
:104E90008289803151F4F8EFCF16FFEFDF06F0E0A2
:104EA000EF06F0E0FF0670F209C088EFC8168FEF3A
:104EB000D8068FEFE8068FE0F80620F281E001C007
:104EC00080E00F900F900F900F90CF91DF911F9186
:104ED0000F91FF90EF90DF90CF90BF90AF909F9099
:104EE0008F9008952F923F924F925F926F927F9290
:104EF0008F929F92AF92BF92CF92DF92EF92FF92EA
:104F00000F931F93DF93CF93CDB7DEB766970FB69E
:104F1000F894DEBF0FBECDBF1C0149875A876B874F
:104F20007C873E872D87DC0115962D913D914D9113
:104F30005C9118972F5F3F4F4F4F5F4F2D833E83FC
:104F40004F835887ED85FE85008111812281338151
:104F5000011511052105310549F048015901089451
:104F6000811C911CA11CB11C10E006C0DC018D90BD
:104F70009D90AD90BC9011E07501640144245524CE
:104F80003201F10185819681A781B08548165906C5
:104F90006A067B0608F09DC02D813E814F815885B1
:104FA0002C153D054E055F0550F4F2E08F2E912C37
:104FB000A12CB12CE2E0CE2ED12CE12CF12CC101A0
:104FC000B701A6019E012F5F3F4F0E949C268823B8
:104FD00009F47FC089819A81AB81BC810097A105CA
:104FE000B10571F08C149D04AE04BF0409F010E00B
:104FF000460157010894811C911CA11CB11C16C0CC
:10500000D701C6010196A11DB11D8B8B9C8BAD8B69
:10501000BE8B88199909AA09BB0929853A854B8550
:105020005C8582179307A407B50759F00894411CC3
:10503000511C611C711C0894C11CD11CE11CF11C89
:10504000A0CF112349F08B899C89AD89BE89F101DC
:1050500080839183A283B383C101B701A6010FEFBF
:105060001FEF2FEF3FE00E942C26882399F431C0D8
:105070002601370108944108510861087108C101EF
:10508000B301A201970186010E942C26882309F111
:10509000730162018C149D04AE04BF0448F3AD8516
:1050A000BE854D915D916D917C91411551056105D4
:1050B000710539F0C101950184010E942C268823D5
:1050C00041F0ED85FE8580829182A282B38281E0EB
:1050D00001C080E066960FB6F894DEBF0FBECDBF6C
:1050E000CF91DF911F910F91FF90EF90DF90CF90C4
:1050F000BF90AF909F908F907F906F905F904F90F8
:105100003F902F900895F999FECF72BD61BDF89A36
:1051100080B50895F999FECF1FBA72BD61BD40BD3B
:105120000FB6F894FA9AF99A0FBE08950F931F9349
:10513000CF93DF93BC018230910510F462E070E000
:10514000E0911F07F091200740E050E0A0E0B0E0C0
:1051500024C08081918186179707D0F08617970722
:1051600071F482819381109729F013969C938E930A
:1051700012972CC09093200780931F0727C04115DA
:10518000510519F08417950718F48D01AC01EF0152
:10519000DF01828193819C01F9013097D1F641159D
:1051A0005105F9F0CA01861B970B8430910580F4F4
:1051B0008A819B810115110521F0F8019383828377
:1051C00004C09093200780931F07FE01329645C0CC
:1051D000FE01E80FF91F6193719302979983888309
:1051E0003CC080911D0790911E07892B41F480914E
:1051F0000C0190910D0190931E0780931D07409123
:105200000E0150910F014115510541F44DB75EB7A4
:1052100080910A0190910B01481B590B20911D07A9
:1052200030911E0724173507B0F4CA01821B930B77
:105230008617970780F0AB014E5F5F4F8417950785
:1052400050F0420F531F50931E0740931D07F90162
:105250006193719302C0E0E0F0E0CF01DF91CF9164
:105260001F910F910895CF93DF939C01009709F44C
:105270008FC0EC0122971B821A8260911F077091E8
:1052800020076115710581F488819981820F931F30
:1052900020911D0730911E072817390739F5D09343
:1052A0001E07C0931D0774C0DB0140E050E0AC173F
:1052B000BD0708F1BB83AA83FE0121913191E20F62
:1052C000F31FAE17BF0779F48D919C911197280FAA
:1052D000391F2E5F3F4F3983288312968D919C9101
:1052E00013979B838A834115510571F4D09320074E
:1052F000C0931F074DC012968D919C911397AD01DD
:10530000009711F0DC01D3CFDA011396DC93CE9332
:105310001297FA0121913191E20FF31FCE17DF07A7
:1053200069F488819981280F391F2E5F3F4FFA0158
:10533000318320838A819B8193838283E0E0F0E044
:10534000DB0112968D919C911397009719F0BC0187
:10535000FD01F6CFAB014E5F5F4FDB018D919C915C
:10536000840F951F20911D0730911E0728173907BC
:1053700079F4309729F41092200710921F0702C089
:10538000138212824250504050931E0740931D07D3
:10539000DF91CF9108956F927F928F929F92AF92FB
:1053A000BF92CF92DF92EF92FF920F931F93CF9312
:1053B000DF938C01009729F4CB010E9496288C0181
:1053C000BBC08EEFE82E8FEFF82EE00EF11E4801E5
:1053D000860E971E8E149F0408F4ACC0D7014D9121
:1053E0005C91119746175707B8F04530510508F4FE
:1053F000A3C0CA0104978617970708F49DC04250BE
:105400005040461B570BF401419351936D937C938D
:10541000CF010E94332990C05B01A41AB50A38015C
:10542000640E751EA0911F07B0912007E0E0F0E028
:10543000CC24DD2447C0A615B705A9F5CD91DC9194
:105440001197CE0102968A159B0568F1CE018A1943
:105450009B09029612962C91129713963C910597F0
:1054600058F0F40122833383CA19DB09D183C08346
:10547000D7016D937C9309C04E5F5F4F4C0F5D1F4A
:10548000F70151834083C901FC01C114D10431F0FB
:10549000D6011396FC93EE9312974EC0F09320071B
:1054A000E0931F0749C08D919C911197E817F90768
:1054B00008F4FC016D0112968C91129713969C9141
:1054C0009C01D901109709F0B6CF80911D079091EA
:1054D0001E0786159705E9F4E617F707D0F4209123
:1054E0000E0130910F012115310541F42DB73EB762
:1054F00080910A0190910B01281B390B82169306AB
:10550000C8F490921E0780921D07F7017183608393
:1055100013C0CB010E949628EC01009759F0D701E7
:105520004D915C91B8010E943802C8010E94332954
:105530008E0102C000E010E0C801DF91CF911F9101
:105540000F91FF90EF90DF90CF90BF90AF909F9022
:105550008F907F906F9008951F920F920FB60F92C9
:1055600011242F933F938F939F93AF93BF93809179
:10557000510690915206A0915306B0915406309175
:1055800055060196A11DB11D232F2D5F2D3720F04B
:105590002D570196A11DB11D2093550680935106EC
:1055A00090935206A0935306B093540680914D06F3
:1055B00090914E06A0914F06B09150060196A11D04
:1055C000B11D80934D0690934E06A0934F06B09365
:1055D0005006BF91AF919F918F913F912F910F9066
:1055E0000FBE0F901F9018958FB7F8942091510619
:1055F0003091520640915306509154068FBFB90125
:10560000CA010895789484B5826084BD84B58160B0
:1056100084BD85B5826085BD85B5816085BDEEE6BA
:10562000F0E0808181608083E1E8F0E01082808199
:1056300082608083808181608083E0E8F0E0808107
:1056400081608083E1EBF0E0808184608083E0EB27
:10565000F0E0808181608083EAE7F0E0808184600F
:10566000808380818260808380818160808380816B
:10567000806880831092C1000895EF92FF920F938B
:105680001F93CF93DF937B018C013FB7F8948091F8
:105690004D0690914E06A0914F06B091500626B54A
:1056A000A89B05C02F3F19F00196A11DB11D3FBF5A
:1056B000BA2FA92F982F8827820F911DA11DB11DE8
:1056C00052E0880F991FAA1FBB1F5A95D1F7EC0112
:1056D00030C00E94C7323FB7F89480914D06909138
:1056E0004E06A0914F06B091500626B5A89B05C066
:1056F0002F3F19F00196A11DB11D3FBFBA2FA92F51
:10570000982F8827820F911DA11DB11D32E0880FAF
:10571000991FAA1FBB1F3A95D1F78C1B9D0B885E62
:105720009340B8F20894E108F10801091109C85141
:10573000DC4FE114F1040105110559F6DF91CF9119
:105740001F910F91FF90EF900895CF93DF93482F13
:1057500050E0CA018A539E4FFC0134914E545E4F73
:10576000FA018491882369F190E0880F991FFC0168
:10577000EC56FE4FA591B491FC01E256FE4FC59147
:10578000D491662351F42FB7F8948C91932F909570
:1057900089238C93888189230BC0623061F42FB7F1
:1057A000F8948C91932F909589238C938881832BE7
:1057B00088832FBF06C09FB7F8948C91832B8C935E
:1057C0009FBFDF91CF910895482F50E0CA018652C4
:1057D0009E4FFC012491CA018A539E4FFC01949173
:1057E0004E545E4FFA013491332309F440C0222312
:1057F00051F1233071F0243028F42130A1F022300F
:1058000011F514C02630B1F02730C1F02430D9F49E
:1058100004C0809180008F7703C0809180008F7DCD
:105820008093800010C084B58F7702C084B58F7DCF
:1058300084BD09C08091B0008F7703C08091B00013
:105840008F7D8093B000E32FF0E0EE0FFF1FE25654
:10585000FE4FA591B4912FB7F894662321F48C9153
:105860009095892302C08C91892B8C932FBF08952A
:10587000682F70E0CB0186529E4FFC012491CB0132
:105880008A539E4FFC0144916E547E4FFB019491CC
:10589000992319F420E030E03CC0222351F1233059
:1058A00071F0243028F42130A1F0223011F514C019
:1058B0002630B1F02730C1F02430D9F404C08091F3
:1058C00080008F7703C0809180008F7D809380005F
:1058D00010C084B58F7702C084B58F7D84BD09C0A8
:1058E0008091B0008F7703C08091B0008F7D80934E
:1058F000B000892F90E0880F991F88559E4FFC01BA
:10590000A591B4918C9120E030E0842311F021E046
:1059100030E0C9010895DC01ED91FC910484F58526
:10592000E02D70E00995089508951F920F920FB62B
:105930000F9211242F933F934F935F936F937F9315
:105940008F939F93AF93EF93FF938091C00082FD5D
:1059500051C0A091C1007091C6004091E6065091DF
:10596000E7064F5F5F4F4F7750708091E806909148
:10597000E90648175907D1F12091E6063091E7066C
:1059800083E0369527958A95E1F78091E606909118
:10599000E706682F6770E091E606F091E706EA5A9D
:1059A000F94F708330E0A1FF0EC0F901EA52F94FC0
:1059B00081E090E002C0880F991F6A95E2F720818C
:1059C000282B20830EC0F901EA52F94F81E090E0C4
:1059D00002C0880F991F6A95E2F780952081822383
:1059E00080835093E7064093E60606C081E08093EB
:1059F000F70602C08091C600FF91EF91AF919F9191
:105A00008F917F916F915F914F913F912F910F9067
:105A10000FBE0F901F901895E0910407F0910507B5
:105A2000E057FF4F8191919120813181821B930B2F
:105A30008F779070892B11F00E94942C08951F92FB
:105A40000F920FB60F9211242F933F934F938F9382
:105A50009F93EF93FF932091F3063091F40680918A
:105A6000F5069091F6062817390731F48091C100A8
:105A70008F7D8093C1003AC0E091F506F091F60663
:105A80008091F5069091F606877021E030E002C023
:105A9000220F331F8A95E2F793E0F695E7959A95E2
:105AA000E1F7F0E0EE50F94F40814223E091F50636
:105AB000F091F606E651F94FE0818091F50690915C
:105AC000F6060196877090709093F6068093F5061F
:105AD0008091C1008E7F8093C100442329F0809182
:105AE000C10081608093C100E093C600FF91EF91F7
:105AF0009F918F914F913F912F910F900FBE0F90DB
:105B00001F901895DC0180E090E01C96ED91FC91CF
:105B10001D97E80FF91F1082019680389105A9F7AB
:105B200080E090E01C96ED91FC911D97E80FF91F25
:105B3000E058FF4F108201968031910599F780E07F
:105B400090E01C96ED91FC911D97E80FF91FEC5623
:105B5000FF4F108201968830910599F71C96ED91C0
:105B6000FC911D97E456FF4F10821C96ED91FC911D
:105B70001D97E057FF4F11821082329611821082DA
:105B80003B961182108232961182108232961082D8
:105B900008958F92AF92BF92CF92DF92EF92FF92D1
:105BA0000F931F93DF93CF93CDB7DEB7FC01138222
:105BB000128288EE93E0A0E0B0E084839583A68310
:105BC000B78382E591E091838083758764875787E7
:105BD0004687318B208B138B028BF58AE48AD78A18
:105BE000C68AB18EA08E828E8E85838F8F85848F9C
:105BF0008889858F8989868FCF010E94822DCF91D8
:105C0000DF911F910F91FF90EF90DF90CF90BF90A9
:105C1000AF908F9008958F929F92AF92BF92CF9244
:105C2000DF92EF92FF920F931F93CF93DF93EC01DC
:105C30007A018B01A22EC22EDD2481E0C822DD2450
:105C4000C8A2BB24403081EE580780E0680780E09E
:105C5000780711F0BB24B39471E0872E912CEA8968
:105C6000FB89BB2069F0C4010E8C02C0880F991F0C
:105C70000A94E2F7808360E079E08DE390E005C06C
:105C8000108260E874E88EE190E0A80197010E941C
:105C90000E3321503040404050405695479537953F
:105CA000279580E12030380720F0BB2011F0BB247D
:105CB000D6CFEE85FF853083E889F9892083EE8988
:105CC000FF898EEFA822A082EC89FD8980818B7FDD
:105CD0008083CD2829F0EC89FD89808184608083D0
:105CE000EC89FD89408121E030E0C9010A8C02C0C5
:105CF000880F991F0A94E2F7482B4083EC89FD89AD
:105D00004081C9010B8C02C0880F991F0A94E2F7E9
:105D1000482B4083EC89FD894081C9010C8C02C06D
:105D2000880F991F0A94E2F7482B4083EC89FD897C
:105D300080810D8C02C0220F331F0A94E2F7209558
:105D400028232083DF91CF911F910F91FF90EF9037
:105D5000DF90CF90BF90AF909F908F900895CF939A
:105D6000DF93DC011C968D919C911D97EC01C3562D
:105D7000DF4FFC01E156FF4F2881398180819181FD
:105D800028173907C9F75496ED91FC915597408132
:105D900021E030E0C9015A960C905A9702C0880F52
:105DA000991F0A94E2F78095842380835496ED919D
:105DB000FC9155974081C9015B960C905B9702C09E
:105DC000880F991F0A94E2F7809584238083549664
:105DD000ED91FC9155974081C9015C960C905C97C0
:105DE00002C0880F991F0A94E2F78095842380836C
:105DF0005496ED91FC91559780815D960C905D973E
:105E000002C0220F331F0A94E2F720952823208333
:105E10001C96ED91FC911D97EE56FF4F808191816C
:105E200092938293DF91CF910895DC011C96ED91BE
:105E3000FC911D97E057FF4F219131918081918115
:105E4000281B390B2F773070C9010895DC011C968F
:105E5000ED91FC911D97EF55FF4F80810895CF93F1
:105E6000DF93AC01FC01A485B585A057BF4F2D91F0
:105E70003C911197A059B040ED01CE56DF4F88817B
:105E800099812817390719F46FEF7FEF24C0E88153
:105E9000F981EA0FFB1F8081682F70E0FA0180A171
:105EA0008823C9F02881398188819981877041E0F0
:105EB00050E002C0440F551F8A95E2F7E3E03695A3
:105EC0002795EA95E1F7A20FB11DA058BF4F8C911D
:105ED000842309F07160CB01DF91CF9108950F9376
:105EE0001F93CF93DF938C01FC01A485B585A05748
:105EF000BF4F2D913C911197A059B040ED01CE5666
:105F0000DF4F888199812817390719F46FEF7FEFE8
:105F100037C0E881F981EA0FFB1F8081682F70E0AC
:105F2000F80180A18823D1F0288139818881998165
:105F3000877041E050E002C0440F551F8A95E2F798
:105F4000F3E036952795FA95E1F7FD01E20FF11D93
:105F5000E058FF4F8081842309F07160FD01EE5607
:105F6000FF4F8081918101968F779070918380831C
:105F7000D8011C96ED91FC911D97EF55FF4F1082B3
:105F8000CB01DF91CF911F910F910895DC015F96B6
:105F90008C915F97882339F05296ED91FC9153973D
:105FA000808186FFF9CF5F961C9208950F931F930F
:105FB000CF93DF93EC018B01AC85BD85A356BF4F1A
:105FC0004D915C911197AD59B0404F5F5F4F477055
:105FD0005070FD01E156FF4F8081918148175907AC
:105FE000D9F388A1882359F1FD01E356FF4F808141
:105FF00091812081318133E0969587953A95E1F73B
:10600000682F70E0277081E090E0382F01C0330FD7
:106010002A95EAF7FD01E60FF71FE456FF4F832F9D
:10602000809590818923808310FF09C0EC85FD85D0
:10603000E60FF71FE456FF4F8081832B8083EC85AA
:10604000FD85E356FF4F80819181ED59F040E80FC7
:10605000F91FEC56FF4F0083EC85FD85E356FF4F9B
:1060600051834083EC89FD89208181E090E00D8C93
:1060700002C0880F991F0A94E2F7282B208381E041
:106080008F8FEA89FB8980818064808381E090E042
:10609000DF91CF911F910F9108958F92AF92BF9290
:1060A000CF92DF92EF92FF920F931F9300D000D018
:1060B000EDB7FEB7319683E0ADB7BEB711968C93BE
:1060C00087E0818385E0828381E0838388EF96E0A7
:1060D00066E576E045EC50E024EC30E000EC10E0C2
:1060E000B1ECEB2EF12CA2ECCA2ED12CF6ECAF2E9B
:1060F000B12CE4E08E2E0E94C92D0F900F900F90CE
:106100000F901F910F91FF90EF90DF90CF90BF9075
:10611000AF908F900895CF93DF930E94022B0E943F
:106120002E0ECCE0DDE20E946C0A2097E1F30E9483
:106130000C2DF9CFCF92DF92EF92FF920F931F9326
:10614000CF93DF937C016B018A01C0E0D0E00FC0E8
:10615000D6016D916D01D701ED91FC910190F08117
:10616000E02DC7010995C80FD91F01501040011536
:10617000110571F7CE01DF91CF911F910F91FF9023
:10618000EF90DF90CF900895DC01ED91FC910190AC
:10619000F081E02D09950895EF92FF920F931F93E0
:1061A0008C01DC01ED91FC910190F081E02D6DE01E
:1061B00009957C01D801ED91FC910190F081E02DD1
:1061C000C8016AE009959C012E0D3F1DC9011F9170
:1061D0000F91FF90EF900895CF93DF93EC0161153D
:1061E000710519F420E030E00FC0DB010D900020B4
:1061F000E9F71197A61BB70BE881F9810280F381BB
:10620000E02DAD0109959C01C901DF91CF91089561
:106210004F925F927F928F929F92AF92BF92CF9256
:10622000DF92EF92FF920F931F93DF93CF93CDB73F
:10623000DEB7A1970FB6F894DEBF0FBECDBF2C011D
:10624000742ECB01223008F42AE019A231E2C32EC9
:10625000D12CCC0EDD1E822E9924AA24BB24672DBE
:10626000752FA50194010E940E3379018A01C8019E
:10627000B701A50194010E94C832472D461B08941E
:10628000C108D1084A3014F4405D01C0495CF601F0
:106290004083E114F1040105110521F07E2C5F2DEE
:1062A000C801DDCFC201B6010E94EC30A1960FB645
:1062B000F894DEBF0FBECDBFCF91DF911F910F913C
:1062C000FF90EF90DF90CF90BF90AF909F908F9016
:1062D0007F905F904F900895DC012115310541F4C6
:1062E000ED91FC910190F081E02D642F09950895C6
:1062F0000E9408310895EF92FF920F931F937C0143
:106300000E946C318C01C7010E94CC309C01200F8F
:10631000311FC9011F910F91FF90EF900895CF9207
:10632000DF92EF92FF920F931F936C017B019A0112
:1063300000E010E0B801A7010E946C318C01C60199
:106340000E94CC30080F191FC8011F910F91FF90B8
:10635000EF90DF90CF900895CF92DF92EF92FF926F
:106360000F931F936C01E62E9A01FF2400E010E0CA
:10637000B801A7010E946C318C01C6010E94CC308B
:10638000080F191FC8011F910F91FF90EF90DF9028
:10639000CF900895CF92DF92EF92FF920F931F93C9
:1063A000CF93DF93EC016A017B012115310541F4A4
:1063B000E881F9810190F081E02D642F09951FC0DB
:1063C0002A303105D1F477FF17C0E881F9810190B7
:1063D000F081E02D6DE209958C0144275527BA0123
:1063E0004C195D096E097F09CE012AE00E9408312F
:1063F0009801280F391F04C02AE00E9408319C012F
:10640000C901DF91CF911F910F91FF90EF90DF9025
:10641000CF900895CF92DF92EF92FF920F931F9348
:106420006C017B019A010027F7FC0095102FB80141
:10643000A7010E94CA318C01C6010E94CC30080F0E
:10644000191FC8011F910F91FF90EF90DF90CF901F
:1064500008950E94EC300895EF92FF920F931F93DE
:106460007C010E94EC308C01C7010E94CC30080FE7
:10647000191FC8011F910F91FF90EF9008950F937E
:106480001F93CF93DF93EC018B016F5F7F4F888168
:1064900099810E94CB29009711F480E005C099836F
:1064A00088831B830A8381E0DF91CF911F910F9135
:1064B0000895CF93DF93EC0188819981892B29F08E
:1064C0008A819B818617970760F4CE010E943F3234
:1064D000882341F08C819D81892B19F4E881F98111
:1064E000108281E0DF91CF910895CF93DF93EC018B
:1064F00088819981009711F00E94332919821882AE
:106500001D821C821B821A82DF91CF910895EF9227
:10651000FF920F931F93CF93DF93EC017B018A01CE
:10652000BA010E945932882321F4CE010E947532AB
:1065300007C01D830C8388819981B7010E944102A5
:10654000CE01DF91CF911F910F91FF90EF900895B1
:10655000CF93DF93EC01198218821B821A821D826D
:106560001C826115710551F0DB010D900020E9F7E7
:106570001197A61BB70BAD010E948732DF91CF9117
:106580000895FC01808191810E9433290895089526
:10659000629FD001739FF001829FE00DF11D649F07
:1065A000E00DF11D929FF00D839FF00D749FF00D93
:1065B000659FF00D9927729FB00DE11DF91F639F34
:1065C000B00DE11DF91FBD01CF0111240895AA1BD3
:1065D000BB1B51E107C0AA1FBB1FA617B70710F0CE
:1065E000A61BB70B881F991F5A95A9F78095909500
:1065F000BC01CD01089597FB092E07260AD077FD2F
:1066000004D0E5DF06D000201AF4709561957F4F25
:106610000895F6F7909581959F4F0895A1E21A2E5F
:10662000AA1BBB1BFD010DC0AA1FBB1FEE1FFF1F36
:10663000A217B307E407F50720F0A21BB30BE40B86
:10664000F50B661F771F881F991F1A9469F76095CD
:106650007095809590959B01AC01BD01CF01089587
:1066600097FB092E05260ED057FD04D0D7DF0AD0A0
:10667000001C38F450954095309521953F4F4F4F71
:106680005F4F0895F6F790958095709561957F4FCF
:106690008F4F9F4F0895EE0FFF1F0590F491E02D4F
:1066A0000994911106C0803219F089508550D0F7B5
:1066B00008959927882708952F923F924F925F92CD
:1066C0006F927F928F929F92AF92BF92CF92DF9202
:1066D000EF92FF920F931F93CF93DF93CDB7DEB767
:1066E000CA1BDB0B0FB6F894DEBF0FBECDBF0994FB
:1066F0002A88398848885F846E847D848C849B8452
:10670000AA84B984C884DF80EE80FD800C811B815F
:10671000AA81B981CE0FD11D0FB6F894DEBF0FBE8E
:10672000CDBFED01089511E0C6EFD1E004C0FE0138
:106730000E944D332296C83FD107C9F7F894FFCF86
:106740005643433A00010101E8038000230700009B
:106750000000B0046009C0128025004B00960000C4
:106760000000B30F820F3B0F440F590F6A0F000058
:1067700000008C159A3039170F17281737150000AD
:106780000000A3179A300000000055239A30000043
:1067900000008B2C9A30152F6F2F2F2FC62FD62F3E
:0267A000262FA2
:00000001FF
